:1000000039C400006FC400006DC400006BC4000060
:1000100069C4000067C4000065C4000063C4000038
:1000200061C400005FC400005DC400000C94AA32EB
:100030000C9464330C945F3255C4000053C4000028
:1000400051C400004FC400004DC400000C9486321F
:1000500049C4000047C4000045C4000043C4000078
:1000600041C400003FC400003DC400003BC4000088
:1000700039C4000005010906A1018506050719E03C
:1000800029E715002501950875018102050719006A
:1000900029EF1500250195F0750181020508190168
:1000A0002905950575019102950175039101C00619
:1000B00060FF0961A1010962150026FF0095207506
:1000C0000881020963150026FF009520750891023A
:1000D000C005010906A101050719E029E71500255A
:1000E00001950875018102950175088101050719BF
:1000F0000029FF150026FF009506750881000508F8
:100100001901290515002501950575019102950133
:1001100075039101C0000000000000000000000015
:1001200000000000000000000000000000000000CF
:100130000000000000000000007E0F00D4FFFFFF61
:10014000C70000007800000000000000002A2B28F3
:10015000000000000000000000000000000000009F
:1001600029000000002C1E342021222434262725BB
:100170002E362D3738271E1F2021222324252633F3
:1001800033362E37381F0405060708090A0B0C0DF5
:100190000E0F101112131415161718191A1B1C1D07
:1001A0002F3130232D350405060708090A0B0C0DE5
:1001B0000E0F101112131415161718191A1B1C1DE7
:1001C0002F3130354C09025B00030100A0FA09040D
:1001D0000000010301010009211101000122440076
:1001E0000705810308000109040100020300000063
:1001F00009211101000122220007058203200001CC
:1002000007050303200001090402000103000000A8
:10021000092111010001223B000705840320000190
:10022000120100020000000870704053010001023A
:1002300003011C037600690061006C003A0066004F
:1002400036003400630032006200330063000000B7
:100250000C0351005500410052004B0000000A03FE
:100260004E006100730070000000040309042900BF
:1002700014001A000800150017001C0018000C00DC
:10028000120013002A002B000400160007000900CA
:100290000A000B000D000E000F0033002800E100E3
:1002A0001D001B000600190005001100100036009B
:1002B000370038003400E000E300E20021522C0057
:1002C0002C002252E7005000510052004F00000065
:1002D000000000000000000000000000000000001E
:1002E00000000000000035001E001F00200021005B
:1002F0002200230024002500260027002A000100F8
:1003000001000100010001000100010001000100E5
:100310002D002E000100E10001000100010001009C
:1003200001000100010001000100010001000100C5
:1003300001000100010001000100010001000100B5
:1003400001000100010000000000000000000000AA
:1003500000000000000000000000000000002E006F
:100360003A003B003C003D003E003F0040004100A1
:100370002F0030004C003900010001000100010095
:100380004200430044004500010031002800010004
:100390000100010001000100010001000100010055
:1003A0000100010001000100010001000100010045
:1003B0000100010001000100010001000100000036
:1003C000000000000000000000000000000000002D
:1003D0000000000000002223252628292A2C2D2F8A
:1003E0003032333536383A3B3D3E4042434547494B
:1003F0004A4C4E5051535557595A5C5E6062646680
:1004000068696B6D6F71737577797B7D7F8183858B
:1004100087898A8C8E90929496989A9C9E9FA1A38D
:10042000A5A7A8AAACAEAFB1B3B4B6B8B9BBBCBEB1
:10043000BFC1C2C3C5C6C7C9CACBCCCDCED0D1D22D
:10044000D2D3D4D5D6D7D7D8D9D9DADADBDBDBDC2F
:10045000DCDCDCDCDDDDDDDDDCDCDCDCDCDBDBDBDB
:10046000DADAD9D9D8D7D7D6D5D4D3D2D2D1D0CE3B
:10047000CDCCCBCAC9C7C6C5C3C2C1BFBEBCBBB940
:10048000B8B6B4B3B1AFAEACAAA8A7A5A3A19F9EBE
:100490009C9A98969492908E8C8A89878583817F86
:1004A0007D7B79777573716F6D6B69686664626067
:1004B0005E5C5A5957555351504E4C4A4947454333
:1004C00042403E3D3B3A3836353332302F2D2C2AD0
:1004D000292826252322FFAA7F554000010101017A
:1004E00001010101010202020202020202020303EF
:1004F00003030303030304040404040404050505BF
:100500000505060606060607070707070808080880
:10051000090909090A0A0A0B0B0B0C0C0C0D0D0D2D
:100520000E0E0E0F0F0F10101111111212131314C3
:1005300014151516161717181819191A1A1B1B1C3B
:100540001D1D1E1E1F202021222223242425262695
:10055000272829292A2B2C2D2D2E2F3031323233CA
:100560003435363738393A3B3C3D3E3F40414243D3
:100570004445464748494A4C4D4E4F5051535455B7
:100580005658595A5B5D5E5F616264656668696B67
:100590006C6D6F7072737577787A7B7D7E808283E5
:1005A0008587888A8C8E8F91939596989A9C9EA029
:1005B000A2A3A5A7A9ABADAFB1B3B5B7BABCBEC036
:1005C000C2C4C6C9CBCDCFD1D4D6D8DBDDDFE2E4FF
:1005D000E7E9EBEEF0F3F5F8FAFDFF1E0F05000476
:1005E0007F3F1F643214643214783C1E1E140A05C7
:1005F0000100010009042D288128000002000200EA
:1006000005042D2881280000030001000A042D287C
:100610008128000004000200EF032D288128BC0A75
:10062000050001000B042D288128000006000200AF
:10063000F1032D28812800000700020007042D285F
:1006400081280000120002000D042D2881280000DE
:10065000130002000F042D2881280000140001005F
:1006600011042D2881280000150000000000C50A93
:10067000D0110000160001000C0444289928000045
:10068000170001010C0444289928000018000102F9
:100690000C044428992800001900020013042D2896
:1006A000812800001A0001030C0444289928000046
:1006B0001B00020015042D2881280000FD377A5800
:1006C0005A000004E6D6B4460200210116000000DC
:1006D000742FE5A3E004C6013C5D003D8889C65443
:1006E00036C3174FE4E5014C7D6CC0F89BB28B47D5
:1006F000216118C274BA6ED506D15248CA509BC740
:100700004F31C4A7663CBD42DB8572B7990644846D
:100710000D0B82DB7C8D28563A5720BF59BA2F85A6
:100720002E04A6B469F8C038972C29569A0F244590
:100730008430E2CAEA69787F48AB349D2B33DF8A84
:10074000AC56D7D98CFA80A1874EF9A65100BAB819
:1007500055A2CFDCAD0F1FC8FD232F428AE9C4414B
:100760007A6A5AFFB57B20867FA6F51F62E2956004
:10077000A30CEC098B5080F13389073B2BFF2CFC39
:10078000C5FF66906D9CD95A5C4D75DA9EBC00DB46
:1007900006F96424D65A1A3DB17F28A19F250B285B
:1007A00012D027A4F4CB8F553B4264650D88D63117
:1007B0006649616208B45B06AC8A8D75BC9AE11328
:1007C000ACD3A393BC41AEC6AE7751ADC16DCCF6F0
:1007D000275B2909D7027D93EE8A0C776CA9CE6D31
:1007E000D152579894E8F7AAC6E53BEA9FB65780DE
:1007F0004A4E47EF428F2AF025B2C3228B0B213E8F
:100800002F99E9884D1AC15389924989AC3B43130A
:100810001C90FA2350C30000264FBB7F0A78023E8B
:100820000001D802C7090000CFF4B3A3B1C467FB2D
:10083000020000000004595A4C4C4C4C4C4C2A52BB
:10084000525252524C4C4C4C4C4C2A5252525252D4
:100850004C4C4C4C4C4C2A52525252524C4C4C4CDC
:100860004C4C2A52525252524C4C004C4C00002AD2
:100870005200525211241FBECFEFD4E0DEBFCDBFD5
:1008800004B603FE18C080911C0490911D04A09131
:100890001E04B0911F048730904BA740B04B59F411
:1008A00010921C0410921D0410921E0410921F043A
:1008B000E0E0F8E3099524E0ACE8B1E001C01D9266
:1008C000AC31B207E1F711E0A0E0B1E0E4E0FCE612
:1008D00002C005900D92AC38B107D9F70E94422AA8
:1008E0000C94CA358DCB9C019A9581159F4118F5C2
:1008F000F32FF270EE27832F8170732F74706627A9
:10090000532F5870442734FF0CC08295807FEF2B03
:1009100009F08062672B09F08064452B69F08068DC
:100920000895EF2B09F08260672B09F08460452B56
:1009300019F08860089580E00895CF93DF93EB016C
:10094000D2DFFE010995DF91CF910895282F92956E
:100950009F70963099F060F4925F9F70923030F4FF
:10096000203FB1F038F481E0283E38F080E008956F
:100970009A5FF3CF81E0243FC9F7089591E0813F6A
:1009800009F090E081E0283E08F080E0892B08958E
:1009900081E008958093A30308958093A4030895AC
:1009A00021E030E001C0220F8A95EAF78091A4038C
:1009B000822BF3CF21E030E0A90102C0440F551F84
:1009C0008A95E2F7CA0180959091A4038923E5CF27
:1009D000382F262F9530A0F58C3090F5892F90E098
:1009E0006CE070E00E94B833830F911D382F377090
:1009F00041E001C0440F3A95EAF733E096958795B8
:100A00003A95E1F763E070E00E94B833FC01E851E9
:100A1000FD4F80E090E0622F70E05191DF019B017B
:100A2000082E02C0369527950A94E2F72170219589
:100A30002527242325272E9301968330910569F7D6
:100A40000895282F953088F58C3078F5892F90E01F
:100A50006CE070E00E94B833820F911DA82FA77040
:100A600023E0969587952A95E1F763E070E00E9470
:100A7000B833FC01E851FD4F40E050E080E02191A7
:100A800030E00A2E02C0369527950A94E2F72170CD
:100A90003327042E01C0220F0A94EAF7822B4F5FFE
:100AA0005F4F4330510559F7089580E008959091C4
:100AB000A40321E030E0F90101C0EE0F8A95EAF7C6
:100AC000D90102C0AA0FBB1F6A95E2F7EA2B01C049
:100AD000220F4A95EAF7892F8E23E81303C0892F46
:100AE000822B5BCF2095822F8923FBCF8091E70259
:100AF00090E020E0022E001C0008281709060CF0E8
:100B000008952F5FF7CFCF93DF93EC01DB018C814A
:100B1000813079F514968C911497813051F5898143
:100B200090E06CE070E00E94B833FC018881E80F2F
:100B3000F11DE85CF74F24912A32D9F011968C917F
:100B4000119790E06CE070E00E94B833FC018C914A
:100B5000E80FF11DE85CF74FE49181E02E1301C02E
:100B600080E091E0EA3209F090E0892BDF91CF91AB
:100B7000089581E0FBCF9C018091A5038D798111BF
:100B800019C0211540E5340780F4211580E23807AB
:100B9000C0F42333310511F1D0F481E02E31310559
:100BA00090F42430310530F00895C901965581152F
:100BB000914010F080E00895C901805F9645079745
:100BC000C8F33327E6CF2C323105A1F70895265319
:100BD000310981E02330310538F3ECCF81E008950D
:100BE0008091AF039091AE03981301C008958F5F79
:100BF0008770FACF9091A903809589238093A903E8
:100C0000282F2770211110C0891771F090911804B6
:100C100092FF0AC0869586958695CCDE1092A90330
:100C20001092AB031092AA030895982F909580918B
:100C3000A50389238093A50308958091A1038115BD
:100C400031F01092A1031092A00310929F03089517
:100C5000803E9105D9F1C8F48133910509F482C031
:100C600048F48932910509F472C08A32910509F479
:100C700080C0089589339105E9F082389105D1F05B
:100C80008533910509F45EC00895843E9105D9F13C
:100C900048F4823E910539F1833E910549F181EE98
:100CA00090E00895863E9105C9F1873E910509F4CB
:100CB0003EC00895209117042370211164C0209133
:100CC000180423FF14C089E290E0089520911704CE
:100CD00020FD45C03091180430FF09C024FD24C018
:100CE00083EE90E008952091170422FDF7CF089538
:100CF0002091170422FD44C03091180430FD43C0F8
:100D000024FFF5CF11C02091180421FFF0CF80916E
:100D1000170484FD09C087EE90E008952091170420
:100D200023FFE5CF24FFF7CF80E090E008952091E6
:100D3000170423FD2BC03091180431FFE1CF84EE5E
:100D400090E008952091170425FFD1CFBCCF2091CA
:100D5000170425FD1EC02091180423FFC8CF89E386
:100D600090E008952091170426FFC1CF8AE290E019
:100D700008952091170426FFBACF81E390E00895EB
:100D800082EE90E0089580EE90E0089586EE90E087
:100D9000089585E390E008959091170492FF10C0A4
:100DA00041E0282F2471243009F040E031E0282F61
:100DB0002871283009F030E0431711F02CE0822729
:100DC00093FF10C041E0282F2471243109F040E046
:100DD00031E0282F2871283109F030E0431711F055
:100DE0002CE082273091180430FF10C051E0282FEA
:100DF0002171213009F050E041E0282F287128307E
:100E000009F040E0541711F029E0822731FF10C0AB
:100E100041E0282F2171213109F040E031E0282FF5
:100E20002871283109F030E0431711F029E08227BA
:100E300094FD877E08951F93CF93DF9309DFEC0124
:100E4000811522E5920708F044C0811540E594071A
:100E500008F0C0C0883E9105E0F4803E910560F442
:100E6000853A910570F4049738F481E0219709F0F0
:100E700080E0C82F50E0D52FCE01DF91CF911F9198
:100E800008958D5C9109D0654397B0F3C0E0D0E040
:100E9000F3CFC11580E4D80798F4C11590E2D907C3
:100EA00008F0AFC0CE019A9581159F4178F78D2F3C
:100EB00073DF182FCE019927CBDEEC01D12BDCCFCD
:100EC000CE019927C5DECC27DF70C82BD92BD06A7D
:100ED000D3CF803842E59407E8F5803652E5950790
:100EE00008F05AC0C03482E5D807E0F4C03292E579
:100EF000D90708F04AC08C2F8695869590E0E5E0EA
:100F0000880F991FEA95E1F7C37021E030E0A9014D
:100F100002C0440F551FCA95E2F7EA01C82BD92B2E
:100F2000DD68AACF8C2F86958695877090E075E056
:100F3000880F991F7A95E1F7C37021E030E0A9018D
:100F400002C0440F551FCA95E2F7EA01C82BD92BFE
:100F5000DC6892CF803C52E5950758F48F71C03A17
:100F6000D24588F590E0982F8827EC01C46FD06AAD
:100F700083CF805C9245809708F088CFDC2FCC2708
:100F8000CC27DF71C06FD06A77CFCF71D0E0DC2F74
:100F9000CC27C16FD06A70CF86958695877090E018
:100FA00045E0880F991F4A95E1F7C37021E030E0D2
:100FB000A90102C0440F551FCA95E2F7EA01C82BE8
:100FC000D92BDA6859CFE8DEC82FD0E0DC2FCC2748
:100FD000D06252CF8F71E0DE93E0CC0FDD1F9A9587
:100FE000E1F7CC27DF70282F30E084FF06C084E0D3
:100FF000220F331F8A95E1F73327C22BD32BD069F9
:101000003BCF8D2F8F71C8DE182FCE01992720DEA0
:10101000EC01D12BDDCF80E00895F894E82FE29524
:10102000EF70F0E041A18F7021E030E0B90102C023
:10103000660F771F8A95E2F7CB01962F9095942340
:1010400091A392A1892B82A3789408950895A0E09A
:10105000B0E0EDE2F8E00C941E34E82FF0E0E55249
:10106000FB4F71110AC0E4912E2F7E2F6E2F822F1D
:10107000CDB7DEB7EAE00C943A34262F30E0C72F24
:10108000D0E04491E42FC42ED12CC90166E070E079
:101090000E94B8338C01EE24EA94F12CC801B70108
:1010A0000E94E233DB01220F331FCB0165E570E0C4
:1010B0000E94B833281B390BA22EAA0CA20EC7011E
:1010C0008C1B9D0BB6010E94B833292FB12CC50192
:1010D000BE010E94B833B701691B7109CB01B6018B
:1010E0000E94B833392FC7018A199B09BE010E949B
:1010F000B833B701691B7109CB01B6010E94B8333F
:10110000792FA330B105B9F00C3F83E0180750F4F4
:10111000A130B105A1F0129709F0A8CFE22F292F35
:10112000742FA4CFA430B10569F0169709F49ECFAF
:10113000722F232F9BCF732FE22F242F97CF742F43
:10114000E32F94CFE92F722FF8CFCF93982F762FDC
:10115000842FC22F692F7BDF472F282F8C2F90E001
:10116000BDD2CF91089580919703843028F4837085
:1011700084608093970308958C3AE8F38370886ABB
:10118000F8CFCF93DF938091970380FD0BC0C0E031
:10119000D0E020E040E060E0CE01A0D22196CE3049
:1011A000D105B9F773D5DF91CF910895FF920F93D1
:1011B0001F93CF93DF93182F062FF42E8091970360
:1011C00080FF0CC0C0E0D0E02F2D402F612FCE015A
:1011D00085D22196CE30D105B9F7D3DFCDB7DEB7B2
:1011E000E5E00C943F34CF93DF93EC0120919A0318
:1011F0009C81892F817090FD822F692F627091FDF3
:10120000622F492F447092FD422FD0DF8C8190E0F5
:101210000196877099278C83DF91CF910895982F3D
:10122000762F842F2091970320FF07C0692F0FDFAF
:10123000962F672F482F892FB9CF0895CF93DF932B
:10124000EC01E7E9F3E0438162818C81E8DF8C8186
:101250008F5F8C83DF91CF910895CF93DF93EC0163
:10126000EC81F0E0EA52FC4F4491E7E9F3E062815F
:101270008181D5DF8C818F5F8C83DF91CF91089541
:101280000F931F93CF93DF93EC0100E010E0802FCA
:1012900062E10E94AF339C81980140919A03609172
:1012A0009903890F52DF0F5F1F4F0E30110579F739
:1012B00068DF8C819A8190FF07C08F5F8C83DF91FC
:1012C000CF911F910F9108958150F8CFEF92FF9227
:1012D0000F931F93CF93DF93FC018281FF24F3943C
:1012E00080FF02C0FF24FA94C0E0D0E020E040E09C
:1012F00060E0CE01F3D104E010E0E12C80915F02C8
:101300008E0D8F309CF16EE00E94D533892F082E10
:10131000001C00088C170D0689F480919A0390E058
:10132000B8010E94B833AC0155954795559547953E
:101330009E01609199038091980307DFEF0C0150A3
:101340001040E1F62196CE30D10581F61ADF80916A
:101350005F02F1E0FF120EC0811591F08150809381
:101360005F02CDB7DEB7E6E00C943E3487FFCFCF07
:10137000825FCDCF90E00196BE010E94F633EFCFA1
:101380008DE0EDCFCF93DF93C0E0D0E020E040E0F0
:1013900060E0CE01A3D12196CE30D105B9F7C0E0EF
:1013A000D0E080915E02082E001C0008C817D0050E
:1013B0005CF180910601082E001C00088C170D06B8
:1013C0001CF19E0140919A036091990380919803CA
:1013D000BCDE2196CE30D10521F7D3DE8091050108
:1013E00090915E02980F90935E0220910601280F63
:1013F00020930601121614F49D301CF08195809301
:101400000501DF91CF91089520E040E060E0CE013A
:1014100065D1DFCFA0E0B0E0E0E1FAE00C941A344F
:101420008C01FC01C481CC2ED12CE12CF12CA70124
:101430009601C701B6010E947335A70196010E946B
:1014400073354B015C0180E290E06C01CC1AD1084D
:101450000D2C000CEE08FF0825E530E040E050E0E0
:10146000C501B4010E9473353B01D82FC92FA701D4
:101470009601C701B6010E947335A70196010E942B
:1014800073359B01AC01280D391D4A1D5B1DB3014D
:101490008D2F9C2F0E94A835D22F822F90E02A32C8
:1014A000B0F563E070E00E94B833AC0197FF02C072
:1014B0004F5F5F4F55954795C42FC095E12CF12C98
:1014C00085E5D82EDD1A8D2DE1FC8D2F97014C2F4F
:1014D000609199033ADE5FEFE51AF50A8EE0E816AF
:1014E000F10489F74EDEF801948181E0911519F03D
:1014F000903219F48FEF8093040180910401890FD9
:10150000F8018483CDB7DEB7EEE00C94363425E5E0
:1015100030E0A901481B590BCA01C3CF0F931F9399
:10152000CF93DF93EC0120E030E06091990380914C
:1015300098039C8189010F5F1F4F273031053CF4D0
:10154000911541F040919A0300DE9801EECF409151
:101550009A03911140E0F9DD98010E30110529F749
:1015600010DE8C8190E00196817099278C83DF9149
:10157000CF911F910F9108958091EF039091F00307
:1015800090931F0180931E010895A0E0B0E0EBEC62
:10159000FAE00C941C34FB018FEF9FEF44305105AF
:1015A00008F467C04091170441FB882780F990E058
:1015B000880F991F42FBAA24A0F8B12CAA0CBB1CCF
:1015C000AA0CBB1C8A299B2940FB882480F8912CFB
:1015D0008829992943FBCC24C0F8D12C53E0CC0CAA
:1015E000DD1C5A95E1F78C299D2944FBEE24E0F897
:1015F000F12C64E0EE0CFF1C6A95E1F78E299F291F
:1016000045FB002700F910E075E0000F111F7A95E7
:10161000E1F7802B912B46FB222720F9C22F20E0F7
:10162000D22FA6E0CC0FDD1FAA95E1F78C2B9D2BC6
:1016300047FB442740F950E05695542F44275795CF
:101640004795842B952B20911804322F3170932BC2
:1016500026952170B22FBB0FA0E08A2B9B2B092E61
:10166000000CAA0BBB0B80839183A283B38380E021
:1016700090E0CDB7DEB7ECE00C94383481E961112D
:1016800001C080E3E82FE295EF70F0E041A18F7098
:1016900021E030E0B90102C0660F771F8A95E2F7BA
:1016A000CB01962F9095942391A392A1892B82A38D
:1016B000089521E9611101C020E3E22FE295EF7066
:1016C000E05EF0E0808190E02F7002C095958795F4
:1016D0002A95E2F781700895509A0895E82F392FDE
:1016E000F62F63E070E00E94B833DC01A351BE4FD7
:1016F0001196FC9311974C938E2F932F63E070E01B
:101700000E94B833FC01E351FE4F22830895AC01DF
:1017100023E0969587952A95E1F78E719927FC012C
:10172000E353FE4F0190F081E02D4F70552721E0EB
:1017300030E002C0220F331F4A95E2F7611541F0F5
:10174000E22BF32B83539E4FDC01ED93FC93089522
:1017500020953095E223F323F5CFFC018481862385
:1017600081110AC082818115B9F06823908593FFA9
:1017700005C081E061110FC080E00895282F2295F7
:101780002F708F70282B962F92959F706F70962BCD
:1017900081E02913F1CF089581E00895E091CD0211
:1017A000F091CE02309739F00190F081E02D309722
:1017B00011F00995089580E00895F0CF0895909173
:1017C0002201913091F0A0E9B1E0EFEF90E02D918E
:1017D000821751F0EF3F19F4211101C0E92F9F5FEB
:1017E0009630A9F7EF3FC9F408959091170497FF39
:1017F000EACFE82FE695E695E695803FA8F7F0E07A
:10180000EA56FE4F877021E030E001C0220F8A9532
:10181000EAF78281822B828308950E2E000CFF0B43
:10182000E257FE4FF8CF90912201913021F4909130
:10183000170497FD0CC0E0E9F1E09191891302C013
:10184000DF011E9251E0E639F507B9F70895E82F58
:10185000E695E695E695803FC8F7F0E0EA56FE4F3C
:10186000877021E030E0A90102C0440F551F8A951E
:10187000E2F7CA018095928189238283089580913D
:10188000210108952FB7F8948091C9019091CA0160
:10189000A091CB01B091CC012FBF08958091F103AD
:1018A0009091F203892B89F0EDDF20919F03309115
:1018B000A003AC01421B530B9A0181E04091F1035C
:1018C0005091F2032417350708F480E00895CF9370
:1018D000DF93C091A5038091A803C82B8091A10339
:1018E0008115E1F08091F1039091F203892B19F0B9
:1018F000D5DF8111A2D9D091A1038091220181303D
:1019000021F48091170487FD13C086E020E931E0BF
:1019100090E0815088F4911190D9CD2B80910303F0
:1019200080958C2390910203892BDF91CF910895AC
:101930008EE128E931E0ECCFF90141919F01411599
:1019400041F39F5FE6CF962F2091180422FF0EC02F
:10195000682F660F660F660F692B6093A90320D866
:1019600091DF9093AB038093AA03089519C89091D7
:10197000A103292F2823211559F0809589238093CD
:10198000A103811531F07EDF80939F039093A00324
:10199000089580E090E0F8CFCF93C82F809118048D
:1019A00082FF0BC08091A1038C1739F06BDF9093FD
:1019B000A00380939F03C093A103CF9108952FB7F5
:1019C000F8946091C9017091CA018091CB01909106
:1019D000CC012FBF0895CF92DF92EF92FF92CF9369
:1019E000DF93D82FC92FC0908103D0908203E0905D
:1019F0008303F0908403E3DF6C197D098E099F094E
:101A0000643F71408105910510F1D9DF6B017C01C4
:101A100082E390E0A0E0B0E0C0927F02D09280022A
:101A2000E0928102F092820280937B0290937C028A
:101A3000A0937D02B0937E02D0937F03C093800376
:101A4000DF91CF91FF90EF90DF90CF90089584EFDA
:101A500091E0A0E0B0E0E0CF08950895FC019B0183
:101A60008091BF019091C0018617970740F0672BC6
:101A700029F48091E8008E778093E800C90140E066
:101A8000009741F4411106C08091E80082FF2EC00A
:101A900080E008952091A6022115A1F12530A1F141
:101AA0002091E80023FD2CC02091E80022FDECCF1E
:101AB0002091E80020FFE4CF2091F20030E0009771
:101AC00019F02830310558F041E02830310509F08F
:101AD00040E02091E8002E772093E800D1CF41919B
:101AE0004093F10001972F5F3F4FE9CF8091A6020D
:101AF000811541F0853041F08091E80083FFC4CF2B
:101B000081E0089582E0089583E008958091B9010D
:101B100087FF13C08091E80082FF06C08091E80033
:101B20008B778093E80008958091A6028111F2CF0F
:101B300008958091A6028115D9F38091E80080FF75
:101B4000F8CF8091E8008E77ECCF2091E4003091BF
:101B5000E50095E6A9012091EC00822F817020FF1D
:101B600006C08091E80080FF06C080E008952091C3
:101B7000E80022FD1AC08091A602811589F0853007
:101B800089F08091EB0085FD0FC02091E400309139
:101B9000E50042175307F9F29A95E1F684E00895BB
:101BA00082E0089583E0089581E00895E091CD02F8
:101BB000F091CE02309739F00284F385E02D309712
:101BC00011F060E209950895982F9093E900891724
:101BD00071F07091EC002091ED005091F00021FD2A
:101BE00009C09F5F953089F78093E9000895762FAB
:101BF000242F50E03091EB003E7F3093EB0030918A
:101C0000ED003D7F3093ED003091EB00316030937B
:101C1000EB007093EC002093ED005093F0002091C6
:101C2000EE0027FDDECF0895CF93A82FB62F209189
:101C3000AF03C091AE032C1303C080E0CF91089591
:101C400030E0C90167E070E00E94B833FC01E05564
:101C5000FC4F81818B1306C080818A1303C085816C
:101C6000841304C02F5F3F4F2770E5CF81E0E6CF9C
:101C70009C012115310509F408958FE99FE0019732
:101C8000F1F700C0000021503109F3CF3BB13E7F96
:101C90002BB121604FB7F8948DEE91E0FC010196D5
:101CA000508168E02BB9000000C057FF3BB9550FC9
:101CB000000000C000C000C03BB900C06A9591F7A9
:101CC00052E08731950751F74FBF8FE594E00197B8
:101CD000F1F700C00000089581E08093E00080E209
:101CE0008093D8001092C9008FE19EE40197F1F72C
:101CF00000C0000087E090EBDC0180931C0490930F
:101D00001D04A0931E04B0931F0488E19CE00FB64D
:101D1000F894A895809360000FBE90936000FFCF69
:101D20000F931F93CF93DF938B01EA019091A6024B
:101D3000943051F58093E9008FEF9091E80095FD84
:101D400006C095ED9A95F1F700008A95B1F780915C
:101D5000E80085FF19C0F9DE811111C08091E8000B
:101D600085FD06C08091E8008E778093E800F3CF70
:101D7000F80181918F018093F100219779F780918B
:101D8000E8008E778093E800DF91CF911F910F914B
:101D90000895792F603229F440E250E0682F82E004
:101DA000BFCF0895CF93DF93D82FC92F48E050E0DD
:101DB000682F792F81E0B4DF88E0ED2FFC2FA1ECB4
:101DC000B1E001900D928A95E1F7DF91CF910895EE
:101DD000BC0140E250E084E0A3CF9091180492FB54
:101DE000222720F9281779F080FB92F990931804A4
:101DF000609117047091180484E090E00E945835B7
:101E000082E00C94FA050895609189038CE090E0DB
:101E10000C943E351F93CF93DF93E82F122F84301D
:101E200008F56530F8F44C30E8F4862F90E068E16E
:101E300070E00E94B833EC01C40FD11DC40FD11D56
:101E40008E2F90E068E770E00E94B833C80FD91F6A
:101E5000632FCE0189960E943E35612FCE018A966E
:101E60000E943E35DF91CF911F910895809122010C
:101E7000813061F58091170487FF28C028DD8093A9
:101E8000970140E250E06DEA72E086E991E00E943D
:101E9000F034892BD1F080E2E6E9F1E0ADEAB2E07E
:101EA00001900D928A95E1F7E091CD02F091CE027A
:101EB000309759F00480F581E02D309731F086E0BD
:101EC0008093960186E991E00995089500DD80935D
:101ED0008E0148E050E06FEC72E08EE891E00E94E5
:101EE000F034892B91F388E0EEE8F1E0AFECB2E05A
:101EF00001900D928A95E1F7E091CD02F091CE022A
:101F0000309719F30280F381E02D3097F1F28EE8DB
:101F100091E0DACF811531F09091A503892B809360
:101F2000A503A4CF0895811531F09091A803892BC2
:101F30008093A8039BCF0895811519F00E94150680
:101F400095CF0895811539F080959091A803892344
:101F50008093A8038BCF0895CF93C82F8115A1F04C
:101F60008238A1F42ADC81FD0FC089E328DC7EDF02
:101F70002FEF87EE93E0215080409040E1F700C0C2
:101F8000000089E350DC72DFCF910895833889F433
:101F900014DC80FDF9CF83E512DC68DF2FEF81EEE2
:101FA00094E0215080409040E1F700C0000083E5BC
:101FB000E9CF843889F401DC82FDE6CF87E4FFDBDA
:101FC00055DF2FEF81EE94E0215080409040E1F703
:101FD00000C0000087E4D6CF8CEF8C0F813A78F5F3
:101FE00080912201813021F48091170487FD0DC07A
:101FF000E0E9F1E086E991E02191C217E1F08E1766
:102000009F07D1F78C2FDBDBBECFEC2FE695E69553
:10201000E695F0E0EA56FE4F828190E04C2F477043
:1020200021E030E002C0220F331F4A95E2F78223FD
:102030009323892B39F38C2FF6DB18DFE3CF80E273
:102040008C0F883008F0A0CFC77021E030E001C0CD
:10205000220FCA95EAF78091A503822B8093A503EE
:1020600092CFCF93DF93EC01805E9109089720F027
:1020700063E97FE0209711F46AE87FE0CE010E94D7
:102080009D048C2F69DFDF91CF910895611529F0B0
:102090002091A80322602093A8039C0130522115AF
:1020A000304308F49927DDCF811559F0823851F477
:1020B00084DB81FF06C089E382DBD8DE89E3B3DB02
:1020C000D5CE0895833841F478DB80FFFACF83E5DD
:1020D00076DBCCDE83E5F3CF843841F46EDB82FF20
:1020E000F0CF87E46CDBC2DE87E4E9CF9CEF980F8A
:1020F000913A28F390E2980F983018F7877091E0A2
:1021000001C0990F8A95EAF7892F0E941506D8CF4A
:10211000CF93DF93EC01C8DFCE01805E9109089771
:1021200020F062EA7FE0209711F46CE97FE0CE01B5
:102130000E949D04DF91CF9108950F931F93CF9339
:10214000DF938C01EB018DDF209739F4C801E0DFCC
:10215000DF91CF911F910F9108958FE99FE0019733
:10216000F1F700C000002197EFCF1F93CF93DF93CB
:10217000182FEB01F1DE209731F4812F95DFDF91ED
:10218000CF911F9108958FE99FE00197F1F700C06B
:1021900000002197F0CF60910F04709110048933F3
:1021A00021F060910D0470910E04DFCFA0E0B0E04B
:1021B000ECEDF0E10C942134E82FF0E0EB5BFE4F06
:1021C000D490282F26952695269530E0F901EB5CD2
:1021D000FE4F0491877010E0082E02C015950795F8
:1021E0000A94E2F701701127F901EB5DFE4FE490CC
:1021F000F12C082E02C0F594E7940A94E2F7E0FA75
:10220000EE24FF24E0F8F901EB5EFE4FC491D0E02C
:1022100002C0D595C7958A95E2F7C170DD270115F3
:10222000110511F081EE98DEE114F10411F086EE53
:1022300093DE60E070E08D2D98DFE114F10411F081
:1022400086EE32DF0115110511F081EE2DDFCD2B69
:1022500011F08CE2A0DFCDB7DEB7E7E00C943D349F
:1022600090918903923061F48A3040F4875F90E066
:102270006AE070E00E94F633875A8DCF8650FDCF1A
:1022800096EF980F963010F0805D90CF895AFDCF71
:10229000CF93DF93EC0188818115D1F08130C1F5B6
:1022A0002981213021F48A81239675DFF4CF2230F1
:1022B00021F48A81239650DEEECF233021F48A81E7
:1022C0002396F2DEE8CF243031F022962111E3CFBD
:1022D000DF91CF9108952A81239680E090E0422FEC
:1022E0004053550BFA014A30510550F0009771F3F5
:1022F000EFE9FFE03197F1F700C000000197F6CF5A
:102300006AE070E00E94B8338E0F9F1F2991E7CFDB
:1023100021964CDFC0CF1092A5038091220181301D
:1023200071F48091170487FF0AC0E8E9F1E08EE1BB
:10233000DF011D928A95E9F71092A80397CDE0E995
:10234000F1E086E0F5CFE7DF2FEF84E39CE021505A
:1023500080409040E1F700C0000088E19CE00FB6AB
:10236000F894A895809360000FBE90936000FFCF13
:10237000CF93DF93D82FC92F2091E702283010F098
:10238000CADF20E0E22FF0E0EE0FFF1FE952FD4F21
:10239000D083C1832F5F2093E702DF91CF9108950F
:1023A000CF93DF93FB018FEF9FEF44305105B0F0E7
:1023B000D081C181B0DFD0931704C370809118041D
:1023C0008C7FC82BC0931804609117047091180477
:1023D00084E090E00E94583580E090E0DF91CF915A
:1023E0000895AAE2B0E0E7EFF1E10C94253489EB1F
:1023F00091E0FC0101962091F100208321E0813CD5
:102400009207B9F78091BA01893009F457C0C8F42E
:10241000823009F4B0C0833009F480C0813081F18A
:102420008091E80083FFE4C08091B9019091BA01E6
:102430009A3008F0DDC0E92FF0E0E453FA4C0C9438
:1024400009348A3009F487C08B3051F78091B90183
:10245000813231F78091BD019091BE01892B01F746
:102460008091E800877F8093E80050DB81E09091C5
:10247000BB01911101C080E0809322014CDFD0CFDD
:102480008091B901813A61F68091E800877F80935D
:10249000E8008091BD019091BE01892B59F060E068
:1024A00080E090E070E0DADA8091E8008B7780934A
:1024B000E800B6CF68E081EC91E0F4CF8091B901FB
:1024C000813209F0ADCF8091BD019091BE018D7F29
:1024D000892B09F0A5CF8091E800877F8093E800E1
:1024E0008091E80082FF15C08091F200823031F4C3
:1024F0008091F100813011F0863021F48091F1005B
:10250000809321018091E8008B778093E800FEDAC8
:1025100087CF8091A6028111E3CF82CF8091B9014C
:10252000813A09F07DCF8091BD019091BE01892B48
:1025300009F076CF8091E800877F8093E800809152
:10254000E80080FFFCCF809122018093F100809110
:10255000E8008E77DACF8091B901813209F060CF3F
:102560008091E800877F8093E800D0DA8091BC01F9
:102570008093200155CF8091B901813A09F050CF65
:102580008091E800877F8093E8008091E80080FFD9
:10259000FCCF80912001D9CF803889F0823841F575
:1025A0008091BD018F70853018F58093E90080918E
:1025B000EB0085FB882780F91092E90006C0809126
:1025C0006F02880F90916002892B9091E800977FAD
:1025D0009093E8008093F1001092F1008091E80060
:1025E0008E7723C0811116C08091BB01813009F123
:1025F0008091E80083FF0AC08091E800877F809384
:10260000E8008091EB0080628093EB00AA96E3E003
:102610000C944134823061F78091BB01811581F0C7
:102620001092E9008091E800877F8093E8006EDADD
:10263000DFCF81E0933009F080E080936F02F0CF2C
:102640008091BD018F702FEF280F243088F6809382
:10265000E9002091EB0020FFE3CF933031F480912B
:10266000EB0080628093EB00DBCF9091EB009061F8
:102670009093EB0021E030E0A90102C0440F551F08
:102680008A95E2F74093EA001092EA008091EB000D
:102690008860E8CF8111ACCF1091BB011F7780918A
:1026A000E3008078812B8093E3008091E800877FAE
:1026B0008093E8002BDA8091E80080FFFCCF8091C6
:1026C000E30080688093E30083E0111101C082E0A1
:1026D0008093A6028DCF8058823008F089CF8091F8
:1026E000BB019091BC018C3D53E0950791F583E0CF
:1026F0008A838AE289834FB7F894DE01139620E03B
:102700003EE051E2E32FF0E050935700849120FF28
:1027100003C082958F703F5F8F708A30C0F0895CF4
:1027200090E08D939D932F5F243161F74FBF80918F
:10273000E800877F8093E8006AE270E0CE010196AE
:102740008DD98091E8008B778093E80051CF805D30
:10275000E7CF292F33272330310509F44EC078F510
:102760002130310509F488C08BE590E0E5ECF1E01B
:102770002230310509F03CCF2091E800277F2093DB
:10278000E8002091BF013091C0018217930708F43F
:102790009C0140E02115310509F073C0411171C061
:1027A0008091E80082FDCDCF8091A602811549F28B
:1027B000853039F28091E80083FFF2CFC2CF80915B
:1027C000BD019091BE012132310509F446C022328B
:1027D000310509F00DCF8330910508F009CFFC01D8
:1027E000EE0FFF1FED5CFE4F0190F081E02D805D4C
:1027F0009E4FDC018C9190E010C09C013327823009
:1028000021F12330310568F4232BB9F4EAE6F2E034
:10281000E4918E2F90E0EAE6F2E0009709F4E8CE2A
:10282000ABCF2330310509F0E3CEE2E3F2E0E491EF
:102830008E2F90E0E2E3F2E0F0CFEEE5F2E0E491FB
:102840008E2F90E0EEE5F2E0E8CFE0E5F2E0E491F3
:102850008E2F90E0E0E5F2E0E0CF8330910508F0C4
:10286000C7CEFC01EE0FFF1FE75CFE4F0190F08129
:10287000E02D89E090E080CF82E190E0E0E2F2E0BC
:102880007BCF8091A602811509F45BCF853009F4D6
:1028900058CF8091E80083FD54CF8091E80082FDFD
:1028A0007FCF8091E80080FF75CF8091F20090E0AB
:1028B0002115310519F08830910550F041E0089755
:1028C00009F040E08091E8008E778093E80062CFC5
:1028D00044914093F1003196215031090196E8CF9F
:1028E000803809F085CE8091E800877F8093E800EA
:1028F000809161028093F10071CE811179CE1091A7
:10290000BB01123008F074CE8091E800877F80937D
:10291000E80010936102FAD81115D9F084E0809391
:10292000A60242E061EC81E04FD942E261EC84E032
:102930004BD942E261EC82E047D942E260EC83E0AD
:1029400043D98091A602843051F482E08093230120
:102950004FCE8091E30087FDE1CF81E0E0CF81E0C1
:10296000F5CF80912501877F809325019091A80361
:102970009D7F9093A80384FF08C08F7E80932501DC
:102980008091A50382608093A5038091250185FF36
:1029900008C08F7D809325018091A503806280937C
:1029A000A50364CACF92DF92FF920F931F93CF9338
:1029B000DF93EC018B01F42E8091250182FF61C031
:1029C000C0908C03D0908D03CC16DD0619F02097B3
:1029D00009F057C0809125018B7F80932501C1E0CC
:1029E00081FD10C080918A0390918B039801281B70
:1029F000390BC1E080911E0190911F012817390702
:102A000008F4C0E080912501C0FB81F98093250185
:102A10006C2FC6010E94870B8091A50381FF08C01F
:102A20008091250180618093250182E00E94150636
:102A30008091A50385FF08C0809125018062809365
:102A4000250180E20E9415066C2FC6011FDBF114E0
:102A500031F080910A0485FF02C086FF25C0809175
:102A60000D0490910E0404D980918C0390918D03F4
:102A70009C0130522115304308F4992749DB71DF5E
:102A80000FC0CE01905281159043B0F4CE0199272A
:102A90003FDB80918C0390918D03C817D90779F3A0
:102AA00010938B0300938A03DF91CF911F910F91B5
:102AB000FF90DF90CF900895CE01EACF1F93CF9380
:102AC000DF93182FA0917D03B0917E03109709F436
:102AD00049C01092800310927F031092030310925A
:102AE00002031696CD91DC911797CE019A95811528
:102AF0009F4108F4D07ED1E0C11101C0D0E0199609
:102B0000ED91FC911A97309731F01B966D917C9165
:102B100080E00995D823D11539F08CEF8C0F813ADC
:102B200028F58C2F0E94130C1115A9F0E0917D035C
:102B3000F0917E03808584FD0EC080917C03811519
:102B400051F0808191819C01215031092F333E4702
:102B500010F40E94EB0C8AD910927E0310927D0330
:102B600010927C03DF91CF911F9108957FD98C2F14
:102B70009BDADACF0F931F93CF93DF930FEE13E01F
:102B8000C9E1D2E0CE010E941D35F80161918F01AB
:102B9000681719F0CE010E943E352196C134F2E04B
:102BA000DF0781F7DF91CF911F910F9108950F9368
:102BB0001F93CF93DF930FEE13E0C9E1D2E0CE0174
:102BC0000E941D35F80181938F012196C134F2E0F6
:102BD000DF07A9F7CAEFD5E0FE018591959100972F
:102BE00011F0FC0109952C96F6E0C63CDF07A1F731
:102BF000DF91CF911F910F910895EFEEF3E0128EC8
:102C0000138E8FEA90E09183808385E0848F28E89B
:102C100033E13383228322E330E0378B268B28ECA9
:102C200030E0318F208F158E35A324A3178E168E9A
:102C300020E530E031A320A382A317A216A29ADFD9
:102C40006ADB109218041092170480E0846080936D
:102C5000180460E074E084E090E00E945835A7CF4B
:102C60000F931F93CF93DF93282F843058F565304F
:102C700048F54C3038F5862F90E068E170E00E940E
:102C8000B8338C01040F111D040F111D822F90E029
:102C900068E770E00E94B833080F191FC8018996D1
:102CA0000E941D35C82FD0E0DC2FCC27C8018A96A2
:102CB0000E941D359E01282BC901DF91CF911F91E4
:102CC0000F91089580E090E0F8CF462F672F209174
:102CD000A9023091AA02232B81F4703F39F4403FBE
:102CE00061F48091A7029091A8020895753028F4AC
:102CF0004C3018F4843008F4B3CF80E090E00895AD
:102D0000A0E0B0E0E6E8F6E10C9421347C0100910B
:102D1000A4038091A303082BC3E0D0E010E0C80116
:102D20000C2E02C0959587950A94E2F780FD09C0A4
:102D30002197A8F7D12C8D2DCDB7DEB7E7E00C9405
:102D40003D34DC2EB7018C2FC0DF0E941B0701979A
:102D500079F3F1CFCF93DF93D82FC92FD1DF6D2F28
:102D60007C2FB3DF0E941B07DF91CF910895FC01F8
:102D70008481811529F080819181ECDF0C94A60477
:102D800080E008951F93CF93DF93182FD92F6115FB
:102D900089F0411579F0B4DFC82F682F812F9D2F5E
:102DA0000E94E804612F7D2F8C2F8FDFDF91CF9160
:102DB0001F9108950E942105C82FF4CFFC01462FD2
:102DC000658180819181DECF382F292FCB01A32F00
:102DD000B22F8F3621E09207A105B10520F48F565E
:102DE0009D4F0C941D3580E0089585E290E00E948F
:102DF0001D358F3089F486E290E00E941D35833ABC
:102E000059F487E290E00E941D3591E08C3C09F076
:102E100090E0892F8170089580E0FCCFAAE0B0E0B7
:102E2000E4E1F7E10C941E3404E013E081E4E82EC1
:102E300082E0F82E97E0B92E27E1C22E22E0D22EB2
:102E4000AA24A3944AE050E0B701CE0101960E9463
:102E50000D35F8013896DF018B2D1D928A95E9F723
:102E600089819A81D80111969C938E938F811296B5
:102E70008C9312978D8113968C9313978885149653
:102E80008C931497898515968C9315978B819C81CB
:102E900017969C938E9316978A8587FD04C01E967D
:102EA000DC92CE921D9780FF02C0F801A08681FFC0
:102EB00007C0D80118969C911897926018969C9319
:102EC00082FF04C0F80190859460908783FF07C05B
:102ED000D80118969C911897986018969C9384FF37
:102EE00004C0F80190859061908785FF07C0D801E4
:102EF00018968C911897806218968C93BAE0EB0E16
:102F0000F11C015F1F4FE1E9EE16E2E0FE0609F059
:102F100099CF2A96EAE00C943A34AAE0B0E0E3E9CB
:102F2000F7E10C941B348090A4029090A50281E0FC
:102F300090E09093A5028093A40200E010E0C80105
:102F40006CE370E00E94B8337C01B12C702E1AC083
:102F500023E0721601F1F601859195919C014A2DAD
:102F60006B2D872D0E940A0FA39432E0C30ED11C53
:102F70008CE0A812EDCFB394ACE0EA0EF11CB5E002
:102F8000BB1661F0C701880F991F9C0122593D4F64
:102F90006901A12CDDCF21E030E0E1CF0F5F1F4FB1
:102FA0000430110561F629DEFE01319689E0DF016A
:102FB0001D928A95E9F78FEF9FEF9E838D8387E0BF
:102FC0008A8701E412E07F014AE050E0B801C701BE
:102FD0000E945C35065F1F4F0139B2E01B07A1F765
:102FE0009092A5028092A4022A96EDE00C943734C8
:102FF000A0E0B0E0EEEFF7E10C941B34FC0182801E
:10300000748081E08483E6EDF3E09490E5E5F4E0FC
:10301000E49100919A030695015810E0000F111FEA
:10302000012F1127C8E1D2E0C12CD12CAA24AA94E7
:10303000B12CE919EE2EF12C83E0881630F4809142
:1030400098038883809199038983711017C01B822C
:103050001A8296014A81698188810E94A5088FEFB2
:10306000C81AD80A25968EE0C816D10429F70E94FE
:10307000C108CDB7DEB7EDE00C9437348B818115F4
:1030800021F181508B8390E06FEF70E00E94B833A4
:103090006C8170E00E94E233FB01FF27EA52FC4F93
:1030A000E491E9198E2F90E06FEF70E00E94B83341
:1030B000B7010E94E23320919A0330E0862F90E01E
:1030C000B9010E94B8339A83C4CF0E94CC34B501B1
:1030D0000E94F633801791070CF0BBCF83E088166F
:1030E00088F00E94CC34B5010E94F63388830E9498
:1030F000CC34209199032695622F70E00E94F6331C
:10310000280F29831A8280919A03893C20F088EC49
:103110008C838B839ECF8431D8F784E1F9CF0F93D2
:10312000CF93DF93C7E9D3E0488159816A817B81DE
:1031300088E090E00E945035288139814A815B8186
:103140006C817D818E819F8100E20E946834622FB4
:1031500083E290E00E943E35DF91CF910F91089578
:10316000E7E9F3E085E0808311828FEF8283838338
:103170001482CF01D4CF80919B03833018F48F5FEA
:1031800080939B0387E993E0CACF80919B038115CD
:1031900019F0815080939B0387E993E0C0CFA0E0B2
:1031A000B0E0E5EDF8E10C941B34182FF62E042F57
:1031B000E22E9091970390FF23C0E92FE695E695C4
:1031C000AE2FB0E0A15CBE4F8C91809395039C7FA5
:1031D0009430D9F4612F7F2D842F0E942708962FD9
:1031E000672F482F892F0E94D60810939803F092DA
:1031F000990300939A03E11419F087E993E08FDFB4
:10320000CDB7DEB7EDE00C943734823019F400917D
:103210009A03EBCF863019F410919803E6CF8930EA
:10322000D9F3893111F7E9518E2F8170782EE69507
:10323000F0E0EA52FB4FE491CE2FD0E0A12CB12C6C
:10324000C12CD12C8EE0882E912CC501B4010E9496
:10325000E233812F711012C0860F9601402F6F2D1F
:103260000E94A5088FEFC81AD80AAC0EBD1E8EE0CA
:10327000C816D10451F70E94C108B7CF861BEDCF05
:10328000E7E9F3E0818121E043816281845F87CFB8
:10329000E7E9F3E0818121E0438162818C507FCFB7
:1032A000E7E9F3E062812CE0620F08F46FEF21E0C0
:1032B0004381818174CFE7E9F3E062812CE0621BF6
:1032C00008F460E021E04381818169CFE7E9F3E020
:1032D00043812CE0420F08F44FEF21E062818181AD
:1032E0005ECFE7E9F3E043812CE0421B08F440E0C5
:1032F00021E06281818153CF9091970390FF2CC090
:10330000811559F18B3258F58F73880F880F909182
:1033100097039370892B80939703611519F087E9C0
:1033200093E0FDDE609197036695669570E04BE053
:1033300050E087E091E00E94E334892B91F01092F5
:10334000960381E08093860220E040919A03609189
:1033500099038091980323CF089581E0D6CF8AE224
:10336000D4CF81E0809396030E94420C9093840214
:1033700080938302E6CF80919703869586958F5F31
:103380008B3208F081E061E0B7CF8091970386959A
:1033900086958A9509F48AE261E0AECFAEE0B0E0AE
:1033A000E4EDF9E10C9416347C01DC0114968C9167
:1033B000811509F46FC160E0C70100DD9C01F701D0
:1033C0008681803170F44091AF039091AE03491330
:1033D00033C09091ED03911521F09091EE0390315F
:1033E00058F1D70115969C91911110C02115B0E5A7
:1033F0003B0708F083C02115E0E23E0708F093C0C8
:10340000283E310590F4203E3105B0F4309301039D
:1034100020930003D70112968D919C919093AD0358
:103420008093AC031092260107C0C9019A958115BB
:103430009F4160F72111EACF61E0C701BFDC8C0139
:10344000F7013580311409F429C197578038910567
:1034500008F0F7C0023008F00CC16EE671E080E0C1
:1034600090E0B2DC811105C1812C912C5401011135
:103470005CC004E0AE014F5F5F4F1A01D101E02F45
:103480001D92EA95E9F724013501FFEF4F1A5F0A13
:103490006F0A7F0AC501B40197DC8983811509F49D
:1034A000E8C0813009F0C9C0A50194012E5F3F4FEB
:1034B0004F4F5F4F2F83388749875A87C301B20127
:1034C00083DC182F8A83811509F4D3C08FEF810F15
:1034D000833008F043C06F81788589859A8574DCD4
:1034E0008B83811519F0C1010E9448112401350117
:1034F00033E0430E511C611C711C6DC0203E42E53F
:10350000340760F4203852E5350708F095CFC9013B
:1035100080529245809708F079CF8ECFC9018757A6
:103520009C470297F8CF8031F6CFFFE68F16F1E087
:103530009F06A104B10409F49CC0C501B40144DC98
:103540002FEF821A920AA20AB20A8111EECF01501D
:103550008ECF4F80588469847A843DC08BEF810F71
:103560008330E0F52401350143E0440E511C611C19
:10357000711C6F81788589859A8526DC8B838115FE
:1035800051F1C301B20120DC8C838115E9F0CB80BD
:10359000DC8051E0C5165FEFD50610F0DC2CCC24A2
:1035A000163079F0173049F0C6010E94EB27809160
:1035B0000D0490910E040E94380EC6010E940C2842
:1035C00003C0C6010E94EB272401350154E0450EDB
:1035D000511C611C711C5301420150CF143009F081
:1035E000B8CF6F81788589859A85EEDB182F240105
:1035F000350164E0460E511C611C711CC501B4010B
:103600006D5F7F4F8F4F9F4FDFDB111591F181155C
:1036100081F18150990B6FEF70E00E94B833A12FB8
:10362000A150BB0B8A0F9B1F0197A8F2EFE9FFE0A7
:103630003197F1F700C00000F7CFC1010E94481197
:10364000CACF0E352CE7120789F00F353CE7130778
:1036500041F00D354CE7140709F5809124018115DF
:1036600029F01092240180E029DA03C081E08093E0
:1036700024018091A9038770811561F0D701159607
:103680008C91811539F08091180482FF03C082E08B
:103690000E94FA052E96E2E10C94323480912401C6
:1036A00081114DC0D70115968C918115C9F0053354
:1036B000FCE71F0709F4D9C108F0C6C103333CE792
:1036C000130709F4CCC104334CE7140709F4CBC148
:1036D00002335CE7150721F4109289030E94040F5E
:1036E000D70115967C90711409F44CC217FF4AC299
:1036F0004801E89497F8A12CB12C0E94DD0B80932F
:10370000880390918903913029F481FF03C089E3F4
:103710000E94CB108091A503809387031092A5038C
:103720001092A80380918903823009F4E5C108F062
:10373000A0C18111D8C182EE0E94AC0FA0C1380196
:10374000B0EE6B1A71085090A2038091A503582A1D
:103750008091A103582AE8E06E16710408F05EC05B
:1037600098012770332781E090E001C0880F2A95E7
:10377000EAF7311409F44FC0582AD7018D919C9172
:103780000E94210521E030E0F90102C0EE0FFF1F89
:103790008A95E2F7FC87EB8720917D0330917E03C9
:1037A00038872F8340918503509186035E874D872C
:1037B00054E0C52E53E0D52EA12CB12C511005C0DC
:1037C000D60112968C9181111BC0F601838190E085
:1037D0002B853C8582239323892B91F08085982F1C
:1037E0009770911101C087E038E06316710408F00A
:1037F00059C0311409F452C086958170811157C0A7
:103800009FEFA91AB90AAFE0CA0ED11CB8E0AB16F7
:10381000B104A1F61CC080955822AFCF31102BC047
:1038200080918503909186030817190781F41092FF
:1038300086031092850310928103109282031092E6
:103840008303109284031092800310927F0380916F
:103850007D0390917E03009709F424CFE8E06E1673
:10386000710408F0DDC0652D0E94AD0B81111ACFE7
:1038700081E024D917CF10938603009385030E941B
:10388000DF0C609381037093820380938303909392
:1038900084031092800310927F036FCF82FB8827EE
:1038A00080F9ACCF311409F4ABCF80FFA9CFD6019A
:1038B0008D909C900815190519F4311409F4A0CFC6
:1038C000EF81F885EC15FD0509F49ACFD6011D9618
:1038D000ED91FC91309721F08081811509F490CF12
:1038E000652DC6010E94AD0B811509F489CF81E0D9
:1038F0000815190509F080E0482E43208114910431
:1039000041F0411006C0ED85FE858E169F0609F038
:1039100077CF80E0D3D8D0927E03C0927D0381E040
:1039200080937C03C5016FE070E00E94B833FC0116
:10393000EC5FFC4F85818093030341100EC081141E
:10394000910459F0808191819C0124503109213AE0
:10395000310508F049C00E94130CC5016FE070E00A
:103960000E94B833FC01EC5FFC4FC680D780C601D3
:103970009A9581159F4110F420EED22299249394B8
:10398000C60101978F339E4708F0912CC5016FE067
:1039900070E00E94B833DC01AC5FBC4F1996ED912A
:1039A000FC911A97309731F01B966D917C9181E0D4
:1039B000099598229114A9F0C5016FE070E00E946A
:1039C000B833FC01EC5FFC4F868197810E94730441
:1039D00080930203C60148E06416710440F40E941B
:1039E000EB0C0E94360F0AC00E945410B6CF049709
:1039F000813A910548F48C2D0E94DF0B411409F4A3
:103A000051CE0E94360F35CE0E94360F8FE39CE9CF
:103A10000197F1F700C000008C2D0E94AC0FEECF93
:103A2000DC012D913C910217130731F4311007C0CE
:103A300010927C0380E01DCF311409F433CEFC01D9
:103A4000808585FD2FCEF6CF06336CE7160779F01B
:103A500007337CE7170709F043CE85E001C081E01A
:103A6000809389033BCE82E0FBCF83E0F9CF84E0F3
:103A7000F7CF843009F454C0853009F456C08FE381
:103A80009CE90197F1F700C000006090890327E0EE
:103A900030E0C901880F991F880F991FB501A40153
:103AA00004C076956795579547958A95D2F74F70DC
:103AB000542EB901615071096B01711451F074E019
:103AC000671219C58AE0481708F415C580E00E94FE
:103AD0003011852D0E94301196019FEFC916D9062D
:103AE000D9F1712CD6CF60910D0470910E0488E14C
:103AF00093E00E949D10C3CF8091880380FD03C096
:103B000083E50E94CB1082EE0E94AC0FEFE3FCE94C
:103B10003197F1F700C0000087E50E94CB10AFCFCE
:103B200086EE0E94CB1088E1F8CF60910D04709171
:103B30000E048BE191E00E949D1060910D04709144
:103B40000E0485E290E00E949D1060910D0470913A
:103B50000E0488E290E0CDCF80918903823009F491
:103B60005FC030F4811151C082EE0E94541006C033
:103B7000843009F45EC0853009F45DC0809187030C
:103B80008093A50380910A0480FF2CC00E94420C00
:103B90005C01D70115968C91811509F4ACC0809118
:103BA000250182FF06C040E0B50180E090E00E9460
:103BB000D2140431BCE71B0709F499C00531ECE7C6
:103BC0001E0709F441C00331FCE71F0709F484C054
:103BD000C80190528115904308F040C010928D03A7
:103BE00010928C03F7019581911509F48CC4809192
:103BF000A5038272F801E052F847EB30F10508F0B6
:103C000046C1EA52FA4C0C9409348CE20E94CB1063
:103C10008091880381FFB2CF89E30E94CB10AECFA1
:103C200082EE0E9454108091880380FDA7CF83E527
:103C3000F4CF88E2F2CF60910D0470910E0488E217
:103C400090E00E949D109ACF90912501892F8E7F40
:103C500090FF8160809325010E94B114809125011D
:103C600080FFC0CF0832110508F05BC00E3111058E
:103C700008F068C0C80104974A9798F580910A0433
:103C800084FD2FC0D70115968C91811509F4BAC017
:103C90009091A5038091A103D82ED92A2D2D2D7F97
:103CA000211509F454C010928D0310928C032091B9
:103CB0000A0421FD4CC060E0C8010E94870B60E04F
:103CC000C8010E9446108091A1038D7F0E94CC0CF8
:103CD00082E00E94FA05CDCC80912501816080931D
:103CE0002501D70115968C91811178CF7BCF8091DA
:103CF00025018E7FAFCF809125018F7E013E11057A
:103D000031F0053E110531F4809125018F7D8093BE
:103D10002501A4CFC80190528115904308F09ECF91
:103D200061CF0933110558F40D32110518F40B3227
:103D30001105B9F680910A0482FDD3CFA3CF0436D2
:103D40001105F7CF80910A0483FDCBCF9BCF27E0ED
:103D5000F701AEE8B3E001900D922A95E1F71092D9
:103D600091031092900380908C0390908D0308151E
:103D7000190591F520910A0425FF2EC030912501E7
:103D800031FBCC24C0F831FF02C026FF25C02091B2
:103D90008A0330918B03F501E21BF30BE83CF1053C
:103DA000D8F491FF08C0809125018061809325019E
:103DB00082E00E9415068091A50385FF08C08091CE
:103DC000250180628093250180E20E9415066C2DFA
:103DD000C4010E9446104DCC8D7F0E94CC0C1093E4
:103DE0008D0300938C03B0928B03A0928A038D2DD8
:103DF0008270846090912501997FD82ED92AD09223
:103E0000250166CF40E0B501C8010E94D21431CC33
:103E10008091970380FF0BC08E7F8093970387E983
:103E200093E07DD9109296030E94C10822CC816054
:103E30008093970361E0869586955EDA1ACC8115AA
:103E400021F0A3DA16CC8115E1F395DA12CC8115B5
:103E500021F01EDA0ECC8115E1F312DA0ACC8115BD
:103E600021F029DA06CC8115E1F31ADA02CC8115AA
:103E700021F037DAFECB8115E1F328DAFACB811590
:103E800021F083D9F6CB8115E1F375D9F2CB073751
:103E9000FCE71F07F9F008372CE7120721F198011A
:103EA000205E32452032310518F5911139C00F716D
:103EB00081E090E0AC0102C0440F551F0A95E2F783
:103EC0008A01642F83E090E00E943E35802F0E949B
:103ED000CA04CFCB81E00E94D00443E062E081E0DD
:103EE0000E945705C6CB82E0911509F412C3F3CFA7
:103EF0009115B1F00A355CE7150709F4CFC008F059
:103F0000A6C001307CE7170709F4C6C003308CE770
:103F1000180709F4BBC001159CE7190709F4A9C0EB
:103F2000F7018581C080D180811509F4BBC0C6012D
:103F30000E948016182F682FC6010E94E804B6015F
:103F4000812F0E9465160E941B07182FD92E86E02C
:103F5000F701DE01119601900D928A95E1F7D701E4
:103F60001596BC9015971696CC90C2949FE0C922E6
:103F70008091A9038770811501F1AB2CB114F1F088
:103F80008D2D807F803461F080E2810F8830A8F031
:103F90008D2D807E803221F4123078F0C11469F0CA
:103FA0008091180482FF09C082E00E94FA05809186
:103FB000A9038770AA24A3948111A12C9D2C92940B
:103FC0008FE09822B8E09B1609F463C1E9E09E16E1
:103FD00008F06DC0F2E09F1608F47DC08EE0890DF8
:103FE0008F70823008F4B2C0492D4850550B4430D0
:103FF000510518F40E94CE0BA12C812F9D2D0E94FB
:10400000A604811541F0B11409F44AC2C11409F49F
:104010003EC210921B04A114A9F08091A90380FD57
:1040200011C0D70115961C928695869586950E949B
:10403000D004C701B3D98091A9038695869586954A
:104040000E94DA0460E0C7010E94DE1623CB0B3524
:10405000ACE71A0729F180911804002482FF039429
:10406000802D0C35BCE71B0709F05ACF0E94ED0EDE
:1040700057CF0E948B11EFEFF4E32CE0E150F040BA
:104080002040E1F700C000000E946C0E6FEF7FEF50
:1040900080E090E00E9458350E94A31181E0E6CFB5
:1040A00080E0E4CFC6010E942105182F48CF29E007
:1040B000921609F45DC186E0890D8F70823008F098
:1040C00093CF123F09F064C18D2D8F71B1105DC186
:1040D0000E94D00489CF0D2D0F7030E1D31610F05F
:1040E0000295007FB114C9F0011569F080E2810FDB
:1040F000883010F011110BC08091A503802B8093A4
:10410000A5030E94360F812F0E94AC0F6DCF8091C6
:10411000A803802B8093A803F4CF812F0E94541012
:10412000011509F461CF80E2810F883010F0111180
:1041300004C0802F0E94150606C000958091A80338
:1041400080238093A8030E94360F4ECF0D2D0F7051
:104150008D2D807F803211F00295007F111549F07E
:10416000113009F475C0B11409F481C0C114E9F02B
:10417000CACF8091180482FD14C0B11459F0011502
:1041800039F08091A503802B8093A5030E94360F00
:1041900080E0BACF80E00E945410011509F424CFCA
:1041A000C8CFB11491F1C11004C0802F0E948A0FB2
:1041B0001BCF51E0C51211C08090A103802F882130
:1041C000081709F411CF0E94420C9093A00380932A
:1041D0009F03802A8092A10307CF80910B04823035
:1041E00008F402CFC81200CF802F0E948A0F802FC0
:1041F0000E94B70C8091A203902F9823091709F40D
:10420000F3CE802B8093A203EFCEC11012C0802F7B
:104210000E949C0F802F0E94B70C8091A203902FC8
:104220009823911509F4E0CE009508230093A2038A
:10423000DBCE80910B04823008F4D6CE61E0C6124A
:10424000D3CE8091A5038023811509F4CDCEDFCF95
:1042500080911104B11421F08C1508F4C5CEA5CFBE
:10426000C81608F0C1CE802F0E949C0FBDCEC1148D
:10427000D1F380910F0490911004193321F08091B3
:104280000D0490910E040E94380E812F0E9454104C
:10429000ABCE8D2D8370811133C0B110A5CE412FCF
:1042A000429546954770440F440F812F8F70042E1E
:1042B00001C0880F0A94EAF7212F207114FF07C06C
:1042C0002FE030E001C0220F4A95EAF720953D2DFE
:1042D000369536953370323071F0333051F040916D
:1042E000A303313029F0822B84230E94CA047CCEA0
:1042F000842B822BFACF822B9091A3038927F5CFB1
:10430000B11459F1D0FE70CE412F429546954770B9
:10431000440F440F812F8F70042E01C0880F0A9420
:10432000EAF7212F207114FF07C02FE030E001C011
:10433000220F4A95EAF720953D2D36953695337034
:10434000323089F0333069F04091A403313041F0CC
:10435000822B84230E94CD0447CE8230A8F644CE1F
:10436000842B822BF7CF822B9091A4038927F2CF45
:104370000D2D0F70B11429F0802F0E94D004812FD1
:1043800015CF812F0E949C0F802F0E94DA042CCE23
:1043900060F4103FB9F0113F81F0B11409F472C01C
:1043A000C110B1CE8D2D8F7193CE133FF9F0143F14
:1043B000A1F78091180482FD25C08D2D8F71B11455
:1043C00021F386CE80911104B11461F0C81608F073
:1043D0000BCE2D2D2F7181E090E001C0880F2A9522
:1043E000EAF7C2CF8C1508F4FFCDF3CF80E0B1140B
:1043F00009F4B0CF81E09D2D9F7101C0880F9A957F
:10440000EAF7A8CF80910B04823048F1B114C9F0CB
:104410009091A9039770943059F41092A9031092C7
:10442000AB031092AA038D2D8F710E94DA04E2CDA6
:1044300063E0C81608F0DECD8D2D8F710E94A30CAD
:10444000D9CDC81640F01092A9031092AB03109278
:10445000AA0364E0F1CF81E00E94FA05CBCDB1144C
:1044600031F063E08D2D8F710E94A30CBDCD81E0F2
:104470000E94FA0572E0C71608F4B6CD82E00E94E9
:10448000FA05B2CDC110F5CE8D2D8F717ECF809102
:10449000A7038093A6038091A5038093A703BBCDB8
:1044A00040E060E089819A810E94C2169C010091DF
:1044B000A503C11429F010921B040093A703ABCDF0
:1044C0008091190490911A0428173907B1F7809147
:1044D0000C0482FFF0CF80911B04811561F3809161
:1044E000A6030E948A0F812F0E94CB108091A60301
:1044F0000E949C0FE0CF5110ECCA243031050CF41F
:10450000E8CA9601C6CA0737BCE71B0709F0C3CC47
:1045100081E00E94DA04E1CC8091EE03803170F4F6
:104520008091ED03811551F02091AF034091AE03CE
:10453000A091E903B091E803421301C0089530E06F
:10454000C90167E070E00E94B833FC01E055FC4F00
:1045500084818115A1F1C90167E070E00E94B83340
:10456000FC01E055FC4F81818A1329C080818B13A7
:1045700026C08581811123C0828193816091EA03E5
:104580007091EB03861B970B883C9105C0F48091DA
:10459000EE038F7080618093EE03C90167E070E0E5
:1045A0000E94B833FC01EA54FC4F90819F709061E7
:1045B000908388EE93E00E94CE190C94F0052F5F53
:1045C0003F4F2770B9CFA0E0B0E0E9EEF2E20C94E3
:1045D0002034D82EC92E0091AF038091AE03081766
:1045E00009F444C010E0C80167E070E00E94B833ED
:1045F000EC0180559C4F7C01FC018581811581F087
:10460000C7010E94B716811559F0CA54DC4F888142
:104610008F7080618883F701808191810E94B81139
:10462000C7010E94CE192091AF0330E02F5F3F4FAA
:10463000277033272093AF03C80167E070E00E9422
:10464000B833FC01E055FC4F81818C11C4CF8081CF
:104650008D11C1CFC80167E070E00E94B833FC0142
:10466000E055FC4F8581811509F4B5CFCDB7DEB794
:10467000E8E00C943C34EF92FF921F93CF93DF93CA
:10468000EC0120912601211541F010E0812FDF91EE
:10469000CF911F91FF90EF900895EA80FB80E61A7A
:1046A000F70A24EFE21621E0F20678F760E0CE0187
:1046B0000E94DE169C0130522115304330F70E94D3
:1046C000BB05811511F380910003909101030E94B5
:1046D000BB05182F8115C9F280911504909116041D
:1046E000853F21E0920710F084EF91E0E816F9068B
:1046F00060F68E818F7080618E83888199810E949F
:10470000B8110E947605CE010E94CE19BFCFADE050
:10471000B0E0EDE8F3E20C9419348C0186E0F80186
:10472000DE01189601900D928A95E1F7D8016C9000
:1047300011965C9011971296AD90BC9013971496B9
:10474000EC9014971596FC90F1100CC05091E70274
:10475000252F30E0E0E08E2F0E2E000C990B8217F3
:1047600093073CF128EEC22E23E0D22E8091EC0379
:10477000811151C0E114D1F0F11409F415C3C8013D
:104780000E94B716811509F40FC36091AC037091B4
:10479000AD03C80170DF811109C087E0F801A8EE00
:1047A000B3E001900D928A95E1F7B6DEFF24F39411
:1047B00088C0880F991F89529D4FDC0111964C913A
:1047C0001197451103C08C91681611F0EF5FC3CFAC
:1047D000EF3F41F2D80116968C9116978F70806149
:1047E00016968C93E517A0F4AFEFA50FA093E70200
:1047F000EA1770F4F0E0EE0FFF1FE952FD4FB0E052
:10480000AA0FBB1FA952BD4F8D919C9191838083AC
:104810000E947605A7CF60E088EE93E00E94DE1646
:104820009C017090ED038091EA039091EB034501A8
:10483000881A990A711409F464C2B8EC8B169104B1
:1048400008F01DC2E11409F4B1CF8091E903F80129
:104850009181E090EE03F0E1EF1608F0D9C19813D2
:1048600059C09091E803D8018C91981353C0F1106E
:1048700051C08E2D8F7080618093EE0388EE93E09F
:104880000E94CE198091EE03F8018683F090EA032E
:10489000E090EB032091AF038091AE03281771F0F5
:1048A00030E0C90167E070E00E94B8338C01005528
:1048B0001C4FD80115968C91811108C00E94F005FB
:1048C000F12C8F2D2D96EFE00C943534C90167E063
:1048D00070E00E94B833FC01E055FC4FC280D380E9
:1048E000C8010E94B71681110EC0C8010E94CE19DE
:1048F0008091AF0390E00196877099278093AF0372
:10490000FC2CED2CC7CF6F2D7E2DC801B4DE81119C
:10491000EFCFD4CF30522115304308F082C0F110D0
:104920000FC140E0652D862D0E94140E81114DC0EF
:1049300040E0652D862D0E94140EF82E811509F495
:1049400033C180910C0480FFBBCF88EE93E00E94BE
:10495000CE1960E088EE93E00E94DE168C01D090C4
:10496000AF037D2C88E0C82E98EE892E93E0992E17
:104970008091AE037816B1F0A72CB12CC50167E089
:1049800070E00E94B833FC01E055FC4F7F0160E00D
:10499000CF010E94DE16582E692ED70115968C91F4
:1049A00081119CC0B8E0CB1608F4C7C088859985F2
:1049B0000ADE0E9476050E94F00587E0E8EEF3E04B
:1049C000DF011D928A95E9F77BCF60E0C8010E9464
:1049D000DE1680910C0483FFABCFB80188EE93E024
:1049E0000E9483058111A4CF8091EE038F708061B6
:1049F0008093EE038091E8039091E9030E94B8113F
:104A000088EE93E00E94CE19E8EEF3E087E0DF0144
:104A10001D928A95E9F788859985D5DD0E947605EE
:104A20004DCFF11409F484CF8091EE03816080931F
:104A3000EE0380910C0481FF43CF88EE93E00E9447
:104A4000CE19F090AF038091AE03F81609F4D8C0E8
:104A50000F2D10E0C80167E070E00E94B833805568
:104A60009C4F0E94B716811509F4CAC0C80167E0BF
:104A700070E00E94B833FC01E055FC4F87E0A8EEDF
:104A8000B3E001900D928A95E1F70F5F1F4F077019
:104A90001127F02E0093AF030E94F0058091AE0322
:104AA0008F1509F40BCF8F2D90E067E070E00E9426
:104AB000B8338C0100551C4FC8010E94B7168111F4
:104AC000FDCEC8010E94CE198091AF0390E00196FF
:104AD00087709927F82E8093AF03E0CF105201150D
:104AE000E0E31E0708F05ECF80910C0483FD0BC04D
:104AF000C72C95012F5F3F4FF22FF7707F2E052DAA
:104B0000162D470135CFB701C4010E9483058115D9
:104B100081F3EECF8D2D90E067E070E00E94B83316
:104B200080559C4F0E94CE198091AF0390E0019672
:104B300087709927D82E8093AF03CD10EBCF36CF57
:104B40008091EE0381608093EE0360E0C8010E94D3
:104B5000DE1680910C0483FF6CCFB80188EE93E0E1
:104B60000E948305811165CFF090EE03E894F0F880
:104B7000F092EE03C8010E94B7168111A1CE8F2DCD
:104B80008F7080618093EE038091E8039091E90338
:104B90000E94B8110E94760588EE93E00E94CE191B
:104BA000E8EEF3E087E00CCF888599850E94AA168D
:104BB000292F22952F70903450F49F70223080F06E
:104BC000911599F0F8019681903178F47ACE2A5FA8
:104BD0002F70223078F0C8010E94CE19F72C71CEC8
:104BE000911519F0811509F46CCE805E883008F4B7
:104BF00068CEF1CF803F08F464CE815F8330F7CF79
:104C000087E0E8EEF3E0DF011D928A95E9F746CFF1
:104C1000981315C09091E803F801808198130FC094
:104C2000F1100DC0E682C8010E94CE1987E0F8019C
:104C3000A8EEB3E001900D928A95E1F7B7CDC801D7
:104C40000E94B716811509F4AFC0F11409F4ACC085
:104C50008091EE03803208F4A0CD8091E80390911A
:104C6000E9039A838983BC82AB828091EC038D83B4
:104C70001E82EF82CE0101960E94CE198ECD9090B9
:104C8000EE03F0E19F1638F488EE93E00E94CE190F
:104C900087E0D60196CEE11409F488CD9091E9031E
:104CA000F8018181981311C09091E80380819813D5
:104CB0000CC0F1100AC09682C8010E94CE1987E08C
:104CC000D6011D928A95E9F771CDC8010E94B716E9
:104CD000811509F469C0F11409F466C08091EE03EE
:104CE000803208F45ACD8091E8039091E9039A83C9
:104CF0008983BC82AB828091EC038D831E829F826C
:104D0000B9CFB8EC8B16910408F052C0E11409F445
:104D10004DCDF11409F448C09091E903F801818167
:104D200098132AC09091E8038081981325C060E011
:104D300088EE93E00E94DE16809113049091140493
:104D40008816990608F072CF8091EE0380FD6ECF31
:104D5000803108F46BCFD80116968C931697982F54
:104D6000907F903F09F45FCF982F907F905F8F7076
:104D7000892B16968C9357CFC8010E94B7168115C0
:104D800071F06091AC037091AD03C80174DC8115C2
:104D900009F403CD87E0E8EEF3E0DF0192CF8091E4
:104DA000EE0381608093EE03C8010E94CE19FECC11
:104DB00087E0F60111928A95E9F782CDABE1B0E088
:104DC000E4EEF6E20C9422344E8B5F8B688F798F81
:104DD000082F8A8F192F9B8FF82EE92E811509F441
:104DE000B8C040E0692F8E899F890E94C2169C013D
:104DF000111549F010921B0490931A048093190422
:104E00001092A8030AC08091190490911A04821785
:104E1000930719F481E080931B041D8A86E0FE014C
:104E20007696DE011F9601900D928A95E1F78091AA
:104E3000180482FF21C08091F1039091F203892B25
:104E4000D9F00E94420C2091AA033091AB03821B3F
:104E5000930B2091F1033091F2038217930738F0FE
:104E60008091A90382FD03C082E00E94FA050E949E
:104E70004E0C81110E941D06F11461F00B8B1C8BEE
:104E800061E0CE010F960E94DE1661E0CE010F9622
:104E90000E94DE160B8B1C8B87E0FE013F96DE0125
:104EA000189601900D928A95E1F7CE0108962FDCB5
:104EB000811126C08091AE034091AF0397E0FE01BF
:104EC0003896DE01119601900D929A95E1F79C8536
:104ED0009115B1F090E09C012F5F3F4F2770332771
:104EE00042171306D1F50E948B111092AE03109257
:104EF000AF0387E0E8EEF3E0DF011D928A95E9F762
:104F00008091AF039091AE03891751F090E067E074
:104F100070E00E94B83380559C4FF9DB811130C09E
:104F20008C85811112C08091260181110EC08A8565
:104F30009B852091AC033091AD03821B930B8F3F77
:104F40009F4318F081E0809326016B96E6E00C9475
:104F50003E34911509F461CF53CF67E070E00E94B1
:104F6000B833DC01A055BC4F87E0FE0131960190BB
:104F70000D928A95E1F72093AE030E94F005C0CF11
:104F80008091AF0390E00196877099278093AF03DB
:104F9000B7CFA6E0B0E0EFECF7E20C9424340E9427
:104FA000420C8C018091AB029091AC02801791076A
:104FB00071F019821A820E94420CBC0149815A8107
:104FC00080E090E0FBDE1093AC020093AB022696EB
:104FD000E4E00C944034A6E0B0E0E1EFF7E20C949A
:104FE00026349093A8028093A702811520E29207AD
:104FF00030F40E9431102696E2E00C94423480EFA7
:1050000089838A830E94420C8160BC0149815A8154
:1050100081E091E0D3DEEFCFA6E0B0E0E2E1F8E29C
:105020000C9426349093A8028093A702811520E265
:10503000920730F40E9488102696E2E00C944234E5
:1050400080EF89838A830E94420C8160BC01498180
:105050005A8181E090E0B2DEEFCF9C01CB01BA0132
:10506000F9013296E4914E2F50E06E17710548F029
:10507000F9013496659175910E94FD3480E090E0CD
:1050800008958FEF9FEF0895A4E0B0E0EAE4F8E21E
:105090000C9423348B01FC013396F49019821A820C
:1050A0001B821C82452B31F48FEF9FEF2496E5E0A5
:1050B0000C943F3444E050E0BE016F5F7F4FCDDF82
:1050C000019691F381E090E00F2C02C0880F991FA8
:1050D0000A94E2F7092E000CAA0BBB0B49815A81F6
:1050E0006B817C8184239523A623B72321E0892B20
:1050F0008A2B8B2B09F420E0F801208380E090E0DC
:10510000D5CF9C01CA01F9013296E4914E2F50E0AF
:105110008E17910558F0F9013496859195910E946A
:10512000FD340E94BA1580E090E008958FEF9FEF64
:105130000895A4E0B0E0EFE9F8E20C941F347C019C
:105140006B01CA01F7013396B49019821A821B824F
:105150001C82892B31F48FEF9FEF2496E9E00C94A9
:105160003B3444E050E0BE016F5F7F4FC70175DF05
:10517000019689F381E090E00B2C02C0880F991F03
:105180000A94E2F780959095092E000CAA0BBB0BB0
:1051900049815A816B817C8184239523A623B7237F
:1051A000F6012081022F017010E00B2C02C0000FCD
:1051B000111F0A94E2F7012E000C220B330B802BF7
:1051C000912BA22BB32B89839A83AB83BC8344E0BE
:1051D00050E0BE016F5F7F4FC70193DFBECFAAE0F3
:1051E000B0E0E5EFF8E20C941A34FE0131968AE063
:1051F000DF011D928A95E9F79AE6A92E91E0B92E72
:105200008F013F01EE24E394F12C3BE7C32E31E004
:10521000D32EF50181915F018F3F09F444C0F894CA
:10522000E82FE295EF70F0E021A18F70A70102C096
:10523000440F551F8A95E2F7CA01922F982B91A32C
:1052400092A18095892382A3789400C0EFE6F1E0D3
:1052500021E030E0812C912C41914F3F79F0A42F37
:10526000A295AF70A05EB0E08C9190E04F7002C04C
:10527000959587954A95E2F780FF3BC080E090E0E6
:10528000882A992A220F331FCE16DF0629F7F50147
:1052900082918F3F11F00E940D0850EA5A95F1F764
:1052A000D8018D929C920E5F1F4FBFE6AB16B1E006
:1052B000BB0609F0AECF4AE050E0B30183E692E0CE
:1052C0000E94F034892BB9F08AE0F301A3E6B2E042
:1052D00001900D928A95E1F781E08093B8010E94D8
:1052E000420C9093B7018093B6012A96EEE00C949D
:1052F0003634C901C5CF8091B8018115B1F3009151
:10530000B6011091B7010E94420C801B910B0597CA
:1053100060F34AE050E063E672E08AE992E00E94BE
:10532000F034892B49F08AE0E3E6F2E0AAE9B2E042
:1053300001900D928A95E1F71092B801D6CFA0E1C5
:10534000B0E0E5EAF9E20C941834FE01319680E110
:10535000DF011D928A95E9F707E110E091E9A92E96
:1053600092E0B92E2FE6422E55245394612C712CD5
:105370004F0173016201B1E14B16510461047104E4
:105380001CF080E1C82ED12CA601B501C4010E94F9
:105390002F35AC0CBD1C0D2C000CEE08FF084C1872
:1053A0005D086E087F080150104019F76096E0E133
:1053B0000C9434346FEF85E290E00E943E356FEF3D
:1053C00086E290E00E943E356FEF87E290E00E9417
:1053D0003E3560E088E290E00E943E350E948D17E5
:1053E000AEDF6FE085E290E00E943E3563EA86E240
:1053F00090E00E943E356CEC87E290E00C943E35E4
:105400008F929F92AF92BF92CF92DF92EF92FF92D4
:105410000F93CF93DF9388E090E00E9425354B01F6
:105420005C01C7E9D3E068839982AA82BB821C82AF
:105430001D821E821F8283E290E00E941D35282F6C
:1054400030E040E050E060E070E080E090E000E2BA
:105450000E944D34282939294A295B292883398318
:105460004A835B836C837D838E839F83DF91CF919F
:105470000F91FF90EF90DF90CF90BF90AF909F90F3
:105480008F900895CDB7DEB7AD970FB6F894DEBF15
:105490000FBECDBF84B7877F84BF0FB6F894A895A1
:1054A00080916000886180936000109260000FBE60
:1054B00080E890E00FB6F8948093610090936100CB
:1054C0000FBE11E0109323018BE098E090938D01C3
:1054D00080938C010E940E170E94D7151092E20053
:1054E0001092E1008091E00081608093E000809163
:1054F000D8008F778093D80019BC809163008160B9
:105500008093630010926202809163008E7F80938B
:105510006300109362021092E2001092E100809109
:10552000D8008F778093D8008091D80080688093CE
:10553000D8008091D8008F7D8093D80084E089BD09
:1055400086E089BD89B5282F21702DA780FFFACF6D
:105550001092A6021092610210926F0210926002E5
:1055600042E060E080E00E94E40D8091E1008E7FE7
:105570008093E1008091E20081608093E20080915D
:10558000E20088608093E2008091E0008E7F80934B
:10559000E0008091E20084608093E2007894809142
:1055A000A602811599F08091E9001091EC008F70AE
:1055B000179511271795182B1092E9008091E80094
:1055C00083FD0E94F1111F701093E90082E084BDF9
:1055D00093E095BD9AEF97BD80936E000E94F516FB
:1055E000811101C0E7DEECE8F2E088E0DF011D9206
:1055F0008A95E9F781E080938B0260E080E00E9469
:105600003E0B61E080E00E943E0BEFE8F1E0319755
:10561000F1F700C0000010E080918B02181708F429
:105620008AC00AE611E0D8018D918D018F3F11F0FB
:105630000E940D08B1E00F361B07A9F70FE611E035
:105640008BE7E82E81E0F82EF80181918F018F3FE2
:1056500011F00E940D08E016F106B1F78AE0EAE9C0
:10566000F2E0DF01282F1D922A95E9F7E3E6F2E048
:10567000DF011D928A95E9F780E090E00E942A35CB
:10568000833E9E4F21F40E94F51681112FC063EED8
:105690007EEF80E090E00E94583560E082E090E08C
:1056A0000E943E3581E08093A30361E083E090E0B7
:1056B0000E943E3560E074E184E090E00E9458353D
:1056C0000E94B01860E08CE090E00E943E3572DEEF
:1056D00040E050E0BA018FE090E00E94503540E099
:1056E00050E0BA0183E190E00E94503582E090E002
:1056F0000E941D358093700284E090E00E942A355C
:1057000090931804809317046ADDEFEFF6E721E029
:10571000E150F0402040E1F700C0000060DD8091E2
:105720009A0280FF1AC06FEF7FEF80E090E00E9446
:1057300058350E946C0E60E0812F0E94590B082F93
:1057400061E0812F0E94590BE12FF0E0E657FD4FF9
:10575000880F802B80831F5F5FCF83E090E00E94E3
:105760001D350E94CA048CE090E00E941D35809394
:10577000890380916D0281111EC087E993E040DEAC
:1057800080919703843028F40E94B01887E993E051
:1057900037DE0E94B308109296030E946C0B809132
:1057A000970380FF05C060E0869586950E947C196E
:1057B00081E080936D0282E191E09093CE0280932C
:1057C000CD028091A60210E406E0853009F48AC07B
:1057D00006DDA1E78A2EA2E09A2EBAE94B2EB2E0AE
:1057E0005B2ED201F401219131918D919D9142E086
:1057F000EB37F40709F480C028173907A1F3FAE959
:10580000AF2EF2E0BF2E10E0D501ED90FD905D01CE
:10581000F401619071904F016E147F0449F16E2480
:105820007F2400E0CC24C394D12CC601862197218B
:10583000892BB1F009831A830E94420C9C838B83CD
:10584000F1E0FD8391E096012E213F21232B09F405
:1058500090E09E8349815A816B817C818D81AEDA93
:105860000F5FCC0CDD1C0C3001F7F401F292E292D8
:105870001F5F153049F60E94DF0C43C08091A602DD
:10588000843019F110926E0288E190E00FB6F8941E
:10589000A895809360000FBE1093600083B7817F4E
:1058A000846083BF83B7816083BF7894889583B712
:1058B0008E7F83BF0FB6F894A895809160008861B1
:1058C00080936000109260000FBE89DCEAE9F2E08C
:1058D00081919191892B09F0A8C5A4EAB2E0AE1795
:1058E000BF07B1F78091A602853009F4C7CF0E94A7
:1058F0008B110E94CE0B6CCF2817390709F07FCF90
:1059000048DBE0907F03F0908003E114F10491F113
:1059100080907F0290908002A0908102B0908202DD
:105920000E94DF0C681979098A099B0980907B0223
:1059300090907C02A0907D02B0907E02681579055F
:105940008A059B05B8F0C7010E94311010928003B0
:1059500010927F0310927F021092800210928102B7
:105960001092820210927B0210927C0210927D02B1
:1059700010927E0280910A0480FF1CC08091250154
:1059800082FF18C00E94420CBC0180918A03909152
:105990008B039B01281B390B80911E0190911F01E5
:1059A0002817390738F041E080918C0390918D03DE
:1059B0000E94D21480919603811509F444C080910D
:1059C0009503E0919703E695E695E81BE093850241
:1059D000853109F49CC008F052C0893009F48DC0AB
:1059E00008F041C0823009F476C0863009F47CC0EA
:1059F00060EDE62E67E0F62E06E218E08091860262
:105A0000811561F0109286020E94420C90938402EC
:105A10008093830210928802109287020E94420CA7
:105A20002091830230918402821B930B8F3F9F470A
:105A300050F42E0D3F1D309384022093830283E89F
:105A400092E0F801099580919402811551F08091BE
:105A50008E021092940280938F0280918C02809328
:105A60008D02E12CA7C08F3019F6E695F0E0ED51DC
:105A7000FA4FE491EE2EF12C06E619E0BFCF54EF79
:105A8000E52EFF24F3940EE81AE0843209F4B6CF31
:105A900090F448E2E42EF12C0AE01AE0883109F48F
:105AA000ADCF833209F0A4CFEEEDF5E0E590F590AF
:105AB00003EF18E0A3CF853209F09ACF8E2F63E071
:105AC00068D6E92FF0E0E552FA4FE491EE2EF12C82
:105AD00008EF17E193CFF0E0E451FA4FE491EE2E96
:105AE000F12C0DE219E08ACFF0E0E751FA4FE49192
:105AF000EE2EF12C0EE119E081CFE695F0E0EA51AF
:105B0000FA4FE491EE2EF12C00E419E077CFF0E0AB
:105B1000E052FA4FE491EE2EF12C02EC19E06ECF38
:105B200061E08E2D0E94590BC82E60E08E2D0E94E0
:105B3000590BCC0C8C292E2D30E0D901A657BD4F26
:105B4000EC919E2F93708917A1F1EE0FEE0FE82BC9
:105B5000EC93EF70F0E0E558FE4F27573D4F808102
:105B6000D9019C91890F8C9384300CF44DC04F2D3A
:105B700050E0BA016F5F7F4F63707727D616170624
:105B800081F044575D4F9E2D9F77FA01948391E0F9
:105B90009F0D937090938E0290918C029F5F9093D3
:105BA0008C02082E000C990B64E070E01FD6F901FE
:105BB0008083E394D0908F02F0908E0280918B02CC
:105BC000E81608F4ADCF90E080918F0220918E020C
:105BD000281779F1E82FF0E0E057FD4F90818F5FB3
:105BE000837080938F0280918D028F5F80938D02EE
:105BF0006AE070E08EE497FD03C06AE070E08BE439
:105C00000E94B5109DA5E0CF8D3F5CF64F2D50E072
:105C1000BA016F5F7F4F63707727D616170609F4B6
:105C2000C0CF44575D4F9E2D9068DA0114969C9327
:105C3000AECF91110E94DF0C0E94CE0B9091950285
:105C4000891721F0809395020E94DF0C8091A602B3
:105C5000843009F0B6CD83E08093E9008091E800BC
:105C600082FFAFCD8091E80090E085FF05C00E94E3
:105C7000A50D811519F19DA58091E8008B77809382
:105C8000E800911509F49DCDE090A902F090AA02D8
:105C9000E981E114F10489F1EE3F09F04FC08A81F6
:105CA000833020F08550833008F048C0EA81EE3020
:105CB00008F044C0F0E0EF51FA4CABC530E2E32EFF
:105CC000F12C9E012F5F3F4F69018091E80085FD17
:105CD0000AC08091E8008B778093E8000E94A50DB0
:105CE000811599F3C8CF8091F100D6018D936D0194
:105CF000B1E0EB1AF10849F7BECFE43148F4E11501
:105D000049F0E150E33130F4F0E0E151FA4C81C563
:105D1000EE3F61F28FEFB4C31A8289E08B830EC02D
:105D20008A81823081F08330B1F0813099F70E940E
:105D3000DF0C75D56B837C838D839E83CE010196AA
:105D40000E94D60D3ECD88E290E077D61B821C8261
:105D50001D828E83F3CF8091A4029091A502892B9E
:105D600069F3FE01319684EA92E0D2012C911196FA
:105D70003C91B2E04B0E511C328323833296841542
:105D8000950599F7DBCF8A81823021F66B817C8182
:105D90008D819E8144D588E290E070D6CFCF4C8132
:105DA0006B818A810E9430169827892798279E83C5
:105DB0008D83C4CF2D813E813227232732274C810A
:105DC0006B818A810E940A0FB9CF0E948D17B6CFCE
:105DD0008A81823891F1B0F48038E9F0813809F095
:105DE000ADCF60E08B810E947C199B8180919703ED
:105DF00091111AC08E7F80939703109296030E9490
:105E0000C1089CCF833809F099CF20E040919A03D4
:105E10006C818B8106C020E04B8160919903809159
:105E200098030E94CF188ACF81608093970360E027
:105E3000869586950E947C1981CF8B8180939B03E8
:105E40007DCF8A818238E1F060F48038A1F081381A
:105E500009F074CF8091970380FF10C086958695D6
:105E60005DCF833809F06ACF809198038B8380914E
:105E700099038C8363CF80919A0350CF80E04ECFFB
:105E800080919B034BCF0E94B30887E993E00E9467
:105E90008F1854CF82E08A8351CF81E08A838FE6C6
:105EA0003DCF0C810D3108F049CF8A809B8098242A
:105EB00089249824A12CB12CFE0131967F010E0F6C
:105EC0001F2F111DE016F10609F438CF80E0FFE620
:105ED0008F16F1E09F06A104B10420F4C4018F568F
:105EE0009D4FABD5D70114968C93BFEFEB1AFB0AED
:105EF000EFEF8E1A9E0AAE0ABE0AE4CF8091A4028A
:105F00009091A502892B09F419CF8C818D3108F06D
:105F100015CF882E912CA12CB12CCA80DB80DC24DB
:105F2000CD24DC24E12CF12C8E010F5F1F4F412C7E
:105F3000512C3201481459046A047B0408F0FECE47
:105F4000FFE6CF16F1E0DF06E104F10438F4D801F2
:105F500014966C91C6018F569D4F90D5BFEF4B1A8A
:105F60005B0A6B0A7B0AEFEFCE1ADE0AEE0AFE0A24
:105F70000F5F1F4FDFCFE3D9E1CE84E08CCF8C8160
:105F80008D3108F0DBCE882E912CA12CB12CCA804B
:105F9000DB80DC24CD24DC24E12CF12C412C512CA1
:105FA00032018E010B5F1F4F481459046A047B04B1
:105FB00008F0C4CE80E0F0EECF16F1E0DF06E10499
:105FC000F10418F4C601899638D5D8018D938D0156
:105FD000BFEF4B1A5B0A6B0A7B0AEFEFCE1ADE0AA1
:105FE000EE0AFE0AE1CF2C81022F10E02D3108F0DD
:105FF000A5CE8A819B819827892798272C01612C1F
:10600000712C803EF1E09F0708F098CE822E912CF3
:10601000A12CB12C40EE51E060E070E0441955092C
:1060200066097709421751056105710508F486CEA6
:106030002091A4023091A502232B09F03EC01C013F
:1060400029E2220E311C80FBEE24FF24E0F880FFC1
:106050000BC08896F2D49D818927982789278115BE
:106060009C4711F48FEF8D83D501C401840D951DDC
:10607000A61DB71D80FF19C0680141E0C41AD108F0
:10608000CE0105968C0D9D1D9CA78BA7C101800F8D
:10609000911FD3D4ABA5BCA59C9181159C4721F43D
:1060A0008FEFEBA5FCA580838601FE013196EE0DF6
:1060B000FF1D2FEFE016F10638F08E010F5F1F4F26
:1060C000C12CD12C760125C09481858181159C47F6
:1060D00011F42483258342E0E40EF11C3296EACFCA
:1060E00080EE481681E058066104710430F4D8014E
:1060F00014966C91C2018996C1D4BFEFCB1ADB0A0A
:10610000EB0AFB0AEFEF4E1A5E0A6E0A7E0A0F5F79
:106110001F4FC814D904EA04FB0410F30FCE80917A
:10612000A4029091A502892B09F408CECE01019614
:106130000E94D60DFFEF21EE34E0F15020403040B8
:10614000E1F700C00000F5CA88E0E7E2F1E0DE0117
:10615000919601900D928A95E1F7FE0132968FE1BA
:10616000DF011D928A95E9F786E0898388E07F96B2
:10617000DE01159601900D928A95E1F7DFCD8CE74F
:10618000898381E08A831B821C82D8CD8B819C818C
:10619000092E000CAA0BBB0B25E0880F991FAA1F24
:1061A000BB1F2A95D1F7AC01BD01405E5F4F6F4F19
:1061B0007F4F481759076A077B0708F4BFCD8C3714
:1061C000E1E09E07A105B10508F0B8CD4D37F1E03B
:1061D0005F076105710520F04CE751E060E070E079
:1061E000481B590BBC016454794FCE010196E2D390
:1061F000A5CD4AE150E06FEF70E0CE01079606D4DE
:106200008091A4028983EA8281E08B831C828D8342
:106210008BE09FCD81E090E09093AA028093A90249
:1062200082E390E090939902809398020E94420C3E
:10623000909397028093960281CDE114F10481F14D
:10624000D0909C02C0909D020091960210919702FE
:106250000E94420C801B910B8536910540F1C3FED4
:1062600026C0D0FE24C00E94420C909397028093D7
:1062700096028091980290919902019790939902C9
:1062800080939802892B61F41092AA021092A902BD
:1062900081E090E09093A5028093A402E12CF12C80
:1062A0008091A4028983EA828091980237CD82E3AB
:1062B00090E09093990280939802F2CF1092A502F9
:1062C0001092A4023BCD0B811C8140E250E06FEFA5
:1062D00070E0CE0101969AD320EF35E042E050E025
:1062E00080E090E0F901659175910617170740F479
:1062F000DE0111968A0F9B1FFC0171836083CA0126
:10630000F6E0203B3F0709F419CDAC014E5F5F4F2B
:10631000245F3F4F4132510528F310CD2B813C8142
:1063200080EF95E0FC01459155912417350709F45C
:1063300098C00C9646E08C3B9407A1F7EBCC8B8180
:106340009C8100EF15E0F8012591359182179307A4
:1063500009F498C0045F1F4FF6E00C3B1F0799F744
:10636000EE24EA94FE2CA9C00E94FD15E7CC8B8197
:10637000853069F0863051F18111E0CC80E2FE0178
:106380003196DF011D928A95E9F788E0C7CC8C81B0
:10639000FE01B1969AE0DF011D929A95E9F78830E7
:1063A00098F490E06AE070E0E3D1BC016F5B7D4F50
:1063B0004AE050E0CF0131D380E089838AE0FE01DA
:1063C000B196DE011296D6CE8FEFF7CF8C819AE090
:1063D000FE013596DE01919601900D929A95E1F7B6
:1063E0002BA13CA12115BCE73B0741F44091A4023D
:1063F0005091A502452B11F420E030E03CA32BA3E3
:10640000883088F490E06AE070E0B2D1BC016F5B44
:106410007D4F4AE050E0CE0181964ED380E08983E3
:106420000E940E178BCC8FEFFACF80916F028115EF
:1064300009F458CAB4E0B9BD09BD09B400FEFDCFE6
:106440008091D8008F7D8093D8008091E000826099
:106450008093E0008091E00081FDFCCF0E948B11D1
:1064600041CAFC013696259135912115310509F473
:1064700051CC4FE150E0BE016E5F7F4FF9010995AD
:1064800089835CCCF8013896259135912115310529
:1064900009F466CF4CE150E0BE016B5F7F4FC8014D
:1064A000F90109957C01892B41F4F8013A9685910F
:1064B0009591009711F0FC010995E9823FCC1F925C
:1064C0001FB61F9211248F939F93AF93BF93809118
:1064D0006E02811113C08091C9019091CA01A091EF
:1064E000CB01B091CC014196A11DB11D8093C90192
:1064F0009093CA01A093CB01B093CC01BF91AF910F
:106500009F918F911F901FBE1F90189578941F9296
:106510001FB61F9211248F939F93AF93BF938091C7
:10652000C9019091CA01A091CB01B091CC01019613
:10653000A11DB11D8093C9019093CA01A093CB0105
:10654000B093CC01BF91AF919F918F911F901FBECF
:106550001F9018951F920F920FB60F9211242F9330
:106560003F934F935F936F937F938F939F93AF93DB
:10657000BF93EF93FF938091E10082FF09C0809168
:10658000E20082FF05C08091E1008B7F8093E100F3
:106590008091E10080FF1AC08091E20080FF16C068
:1065A0008091E2008E7F8093E2008091E200806122
:1065B0008093E2008091D80080628093D80019BC5B
:1065C00085E08093A60283E0809323018091E1001F
:1065D00084FF2FC08091E20084FF2BC084E089BD3E
:1065E00086E089BD09B400FEFDCF8091D8008F7D83
:1065F0008093D8008091E1008F7E8093E1008091AC
:10660000E2008F7E8093E2008091E20081608093BF
:10661000E20080916102811509F44CC084E080930E
:10662000A6028091A602843009F04CC082E08093DB
:1066300023018091E10083FF2CC08091E20083FF61
:1066400028C08091E100877F8093E10082E0809301
:10665000A602109261028091E1008E7F8093E1009A
:106660008091E2008E7F8093E2008091E200806161
:106670008093E20042E060E080E00E94E40D8091BF
:10668000F00088608093F00081E080932301809384
:106690002201FF91EF91BF91AF919F918F917F91D7
:1066A0006F915F914F913F912F910F900FBE0F907F
:1066B0001F9018958091E30087FF02C083E0AFCF61
:1066C00081E0ADCF81E0B3CF1F920F920FB60F9252
:1066D0001124EF92FF920F931F932F933F934F93A9
:1066E0005F936F937F938F939F93AF93BF93CF935A
:1066F000EF93FF9309EE10E0F8018081C091EC0068
:106700008F70C795CC27C795C82B108280EFE82ED5
:10671000F12CF7018081877F808378940E94F111AA
:10672000F8011082F701808188608083CF70F801C2
:10673000C083FF91EF91CF91BF91AF919F918F91C6
:106740007F916F915F914F913F912F911F910F9189
:10675000FF90EF900F900FBE0F901F9018950024A0
:1067600080FD060E660F11F08695D1F7802D0895F5
:106770000024552704C0080E591F880F991F009741
:1067800029F076956795B8F37105B9F7802D952FA7
:106790000895992778E0880F991F961708F0961B9F
:1067A000881F7A95C9F78095089587FB082E0626DD
:1067B00087FD819567FD6195ECDF0EF4919507FCEF
:1067C00081950895AA1BBB1B51E107C0AA1FBB1FDF
:1067D000A617B70710F0A61BB70B881F991F5A956D
:1067E000A9F780959095BC01CD01089597FB072EE0
:1067F00016F4009406D077FD08D0E4DF07FC05D03E
:106800003EF4909581959F4F0895709561957F4FC7
:106810000895EE0FFF1F0590F491E02D099469276C
:106820009627692778278727782708952F923F9200
:106830004F925F926F927F928F929F92AF92BF9290
:10684000CF92DF92EF92FF920F931F93CF93DF933C
:10685000CDB7DEB7CA1BDB0B0FB6F894DEBF0FBE99
:10686000CDBF09942A88398848885F846E847D84E6
:106870008C849B84AA84B984C884DF80EE80FD80E8
:106880000C811B81AA81B981CE0FD11D0FB6F8945E
:10689000DEBF0FBECDBFED010895002E083090F091
:1068A000982F872F762F652F542F432F322F222793
:1068B0000850F4CF220F331F441F551F661F771F48
:1068C000881F991F0A95B2F7002D089597FD10941F
:1068D000002E083098F00850232F342F452F562FC4
:1068E000672F782F892F912DF4CF15949795879541
:1068F0007795679557954795379527950A95AAF700
:106900001124002D08958F929F92AF92BF92CF9243
:10691000DF92EF92FF92CF93DF93EC016881798150
:106920008A819B81611571058105910521F464E2DD
:1069300079ED8BE597E02DE133EF41E050E0ECD0CD
:1069400049015A0127EA31E440E050E0CCD06B0124
:106950007C012CEE34EF4FEF5FEFC501B401C3D0E3
:10696000DC01CB018C0D9D1DAE1DBF1DB7FF03C00B
:106970000197A109B04888839983AA83BB839F7735
:10698000DF91CF91FF90EF90DF90CF90BF90AF90CD
:106990009F908F900895B7CF80E091E0B4CFA0E0B2
:1069A000B0E08093000190930101A0930201B093A5
:1069B00003010895FB01DC0102C005900D924150D6
:1069C0005040D8F70895FC014150504030F00190FC
:1069D0000616D1F73197CF01089588279927089592
:1069E000FB01DC0104C08D910190801921F441501C
:1069F0005040C8F7881B990B0895FB01DC0102C0C9
:106A000001900D9241505040D8F70895DC0101C02B
:106A10006D9341505040E0F70895DC01CB01FC013B
:106A2000F999FECF06C0F2BDE1BDF89A319600B4E7
:106A30000D9241505040B8F70895F999FECF92BD9C
:106A400081BDF89A992780B50895A6E1B0E044E0A9
:106A500050E0E5CFA8E1B0E042E050E0E0CFDC015B
:106A6000A40FB51F4150504040F0CB01840F951F3B
:106A70002E9105D041505040D8F70895262FF9990E
:106A8000FECF92BD81BDF89A019700B4021639F08D
:106A90001FBA20BD0FB6F894FA9AF99A0FBE08955E
:106AA0000396272FECDFEADF252FE9DF242FE7CF3E
:106AB0000196272FE4DFE2CFDC01CB0102C02D914C
:106AC00005D041505040D8F70895262FF999FECFB0
:106AD0001FBA92BD81BD20BD0FB6F894FA9AF99AFB
:106AE0000FBE01960895EE27FF27AA27BB2708C0EF
:106AF000A20FB31FE41FF51F220F331F441F551FA2
:106B0000969587957795679598F37040A9F70097C4
:106B100099F7BD01CF010895052E97FB16F4009457
:106B20000FD057FD05D014D007FC02D046F408C0A2
:106B300050954095309521953F4F4F4F5F4F0895A9
:106B400090958095709561957F4F8F4F9F4F0895D9
:106B5000A1E21A2EAA1BBB1BFD010DC0AA1FBB1F61
:106B6000EE1FFF1FA217B307E407F50720F0A21BD3
:106B7000B30BE40BF50B661F771F881F991F1A9440
:106B800069F760957095809590959B01AC01BD016A
:106B9000CF010895F894FFCFCC12F212F812F2123E
:106BA000F8124A136B13F81270147D14081F1F1F7C
:106BB000231F271F2B1F2F1F331F371F3B1F3F1F55
:106BC000431FA430BF30C6309E2E9E2EF9300A31AE
:106BD0001D315E3163318E319F31B431B7318C2E2E
:106BE000902EC32ECF2EDA2EE52EE82E212F432F06
:106BF0008A2E8F304A2F4D2F512F7E2FBB2FBD2F26
:046C0000BF2FF32F80
:106C04000100000001010201191A1B1C1D1E1F2096
:106C140021223F0CD20EE80E2C0D2D0DC90EAF0013
:106C24000000010001010180052436EA8520780076
:106C340044223BD100AF007400D701F001100200E0
:106C440001020202020606060909090909090F0FD1
:106C54000F0F0F0F151515181919191919191919D5
:106C640019192324252525252525656466673734C8
:106C7400353633623296929394953100FF010001C8
:0C6C84000000FFFF0000010001FF000005
:00000001FF
